:10200000008000208D260000752600007526000047
:1020100000000000000000000000000000000000C0
:102020000000000000000000000000007526000015
:10203000000000000000000075260000E1260000FE
:102040007526000075260000752600007526000024
:102050007526000075260000752600007926000010
:102060007526000075260000752600007526000004
:102070007526000075260000E52500007526000085
:10208000752600007526000075260000A1230000BB
:10209000000000007526000075260000752600006F
:1020A00075260000752600007526000075260000C4
:1020B0000000000010B5064C2378002B07D1054B1B
:1020C000002B02D0044800E000BF0123237010BDA4
:1020D000100200200000000028940000044B10B5FE
:1020E000002B03D00349044800E000BF10BDC046E8
:1020F000000000001402002028940000002370B5A6
:102100000E4C23602168B42908DC0D4800F048FA21
:102110000F2000F029FB23680133F2E7094D0A493B
:10212000280002F0EFFB0A222168280002F049FC97
:102130002800064902F0E6FB70BDC04634020020CC
:102140002C02002018050020D78C000041910000CF
:10215000B42370B50E4C23602168002908DB0D48BC
:1021600000F01EFA0F2000F0FFFA2368013BF2E7AF
:10217000094D0A49280002F0C5FB0A2221682800FF
:1021800002F01FFC2800064902F0BCFB70BDC046EF
:10219000340200202C02002018050020BC8C000016
:1021A0004191000010B5234B88B01868C0B200F010
:1021B00067FC214C206004F017FC00221F4B03F049
:1021C00007FE00221E4B03F003FE0B00022102005B
:1021D000009102A802F079FC02A905A802F060FCB7
:1021E000184905A802F0C4FC0100174802F09CFB46
:1021F00005A802F0EAFB02A802F0E7FBFA20400083
:1022000000F0B2FA206804F0EFFB00220B4B03F061
:10221000DFFD00220D4B02F08DFE002807D0FFF7F6
:102220006DFFFA20C00000F09FFA08B010BDFFF764
:102230008FFFF6E700000020300200200000503F32
:1022400000005940F18C0000180500200000E03F1C
:1022500010B5024800F0AEF810BDC0462C020020B8
:1022600010B50921044800F06BF996210348890153
:1022700000F0F2FE10BDC0462C0200201805002020
:10228000F7B50C27404E0193335C04005BB20D00A0
:1022900000924743002B2EDA00230B82EB7BDB09F5
:1022A000FCD1335D394A01335BB23355335D12786B
:1022B0005BB2DB19934203DA335D5BB20B2B34DD87
:1022C0002F8ABFB2EB7BDB09FCD1314B3149186857
:1022D00002F0A4FC304B04375843009B00090C3338
:1022E00087424DD280B25B005853EB7BDB09FCD1B7
:1022F000FF33335540E0335C244A5BB21278DB197C
:102300009342CEDA335C254A5BB2DB19DB009B5C7F
:102310005B06C6D5335C00215BB2DB19DB00985C41
:102320008006800E00F066FCBBE7335D1B4A5BB2A3
:10233000DB19DB009B5C5B0609D5335D01215BB2D9
:10234000DB19DB00985C8006800E00F053FC2A8AC3
:1023500092B2EB7BDB09FCD1335D5BB2DF190F4B33
:10236000FF00DF197B68D318009A9BB20C32520031
:102370005353EB7BDB09FCD16B461B79AB73F7BD89
:10238000BFB25B005F53B0E7390200203802002083
:102390000400002040420F00204E00003C020020BC
:1023A000002210B5102302491000FFF769FF10BD8D
:1023B0000030004270B50C4B05001C780B2C10D877
:1023C000621C1A70094B04701868094902F026FC57
:1023D000084BE4005843084B00091C1960602800B2
:1023E00070BDFF230370FAE73802002004000020CC
:1023F00040420F00DC0500003C020020F7B50193CD
:10240000037804000E0017000B2B00D986E0C8B239
:10241000012100F0A3FB3F2132002078404DC30092
:102420005E5D0A408E4316435E5588230322962143
:102430009B00DB1BDF171740FF18019B0901C91A1E
:10244000CB1713405B189B10BF10A37067700C2153
:1024500002F0E4FB0C23C0B243431A000C32D90053
:10246000695C490654D401339342F8D100284FD116
:102470002C4B2D4A5A805A78D209FCD12B4E02326D
:10248000338893433380F37BDB09FCD10133338002
:10249000F37BDB09FCD13388DB07FCD433889BB2A8
:1024A0003380402332881343338080233288DB001B
:1024B000134333800123327913433371F37BDB09F8
:1024C000FCD11B4B1B49186802F0A8FB0300FA2043
:1024D00080005843000980B23083F37BDB09FCD1D4
:1024E0008021154B0903D967C023C420134A5B0020
:1024F000D150800013581B021B0A13501023116087
:10250000737332880E3B13433380F37BDB09FCD1BA
:1025100040222378DB00E95C0A43EA542078FEBDC0
:102520003C020020000C00401C4000000030004233
:102530000400002040420F0004E100E000E100E060
:102540009623882210B51B019200FFF757FF10BD9C
:1025500070B505780B2D1BD801238824C356E41AC7
:10256000A4008C4208DC96248078A40040B2241A8F
:10257000A4008C4200DD0C00064B0749186802F0ED
:102580004DFB053C6043054BED0000095D1968609B
:1025900070BDC0460400002040420F003C020020F5
:1025A0000F4B13B50400994216DCB420B42902DCA9
:1025B000C843C017084001228823A25602219B1A53
:1025C000962261569200521A9200009200219B00BE
:1025D000B42202F0D9F801002000FFF7B9FF13BDC3
:1025E0001F02000010B5024802F013F810BDC046EB
:1025F0009C02002013B51249124800F0D5FB124985
:10260000124800F0D1FB1249124800F0CDFB1249EC
:10261000124800F0C9FB1249124800F0C5FB124CE9
:102620001249200000F0C0FB012301930233009304
:102630000D220B3321000E4801F064FF13BDC0468C
:1026400000080042E0040020000C0042E8040020E2
:1026500000100042F004002000140042F8040020A2
:10266000001800420005002008050020001C004260
:102670009C020020FEE70000034B10B51B68002BF6
:1026800000D0984710BDC0461005002070B50F4916
:102690000F4CA14204D100F08FF802F079FAFEE766
:1026A0000C4D00238D42F6D0CA18E818A24205D37B
:1026B000094B8242EFD00949002204E0006804334C
:1026C0001060F1E704C38B42FCD3E4E70000002074
:1026D000100200202C94000010020020500B00205B
:1026E00010B500F066F8002801D100F057F810BDD1
:1026F000014B18607047C04610050020014B186858
:102700007047C04614050020F7B5134801228446DF
:102710001249134C8E68636805689B0E1340019242
:1027200088686268019F920E3A4067463F6893420C
:102730000ED1BD420CD186420AD35B19FA254868F6
:10274000AD00861B07486B437043000DC018FEBDEB
:102750003D0013000600E3E71405002010E000E050
:1027600000ED00E05555000070B5041E10D0FFF7D5
:10277000CBFF050000F01CF8FFF7C6FF054B401B20
:102780009842F7D9FA23013C9B00ED18002CF3D1B5
:1027900070BDC046E70300007047000010B5034A53
:1027A00013680133136000F0C3FA10BD1405002054
:1027B00070470020704700001E2270B54648474908
:1027C000436893431C3A1343436008238C692343B3
:1027D0008B61434C434B9C829C8A14439C82DC68F3
:1027E0001442FCD00124404A14701578254203D0CD
:1027F00055786DB2002DF8DB01249460547864B2F2
:10280000002CFBDB394C5460547864B2002CFBDBA9
:102810008224E4015480547864B2002CFBDB02244F
:102820009C840E34DD682542FCD0314CDC621024DF
:10283000DD682542FCD09D8C2E4C2C439C841024BA
:10284000DD682542FCD002249D8C80262C439C848C
:102850004024DD683542FCD0DD682542F9D01024E3
:10286000DD682542FCD000249460547864B2002CCA
:10287000FBDB214C5460547864B2002CFBDB1C6AF7
:102880001E4D2C4080251C621C6AAC431C62032335
:1028900093601B4B536053785BB2002BFBDB002330
:1028A000FF240B72174A4B728B72CB72164B1A6055
:1028B000164B174A1B6811689A065B01C90E234024
:1028C000520F12020B431343124A138580234268AE
:1028D0001343436070BDC046004000410004004007
:1028E0000C06000000080040000C0040010501003B
:1028F000B905FF7D040A000000070300FFFCFFFF8D
:1029000003060100006CDC0204000020246080004B
:102910002060800000400042FA21314B10B5186859
:10292000890002F07BF92F4B0138984256D82E4986
:102930002E4A4860C020136A00061B021B0A03438C
:102940001362002407238C600B608021136A090640
:102950001B021B0A0B431362FC22254B196A0A4314
:102960001A62FC22196A92010A431A62A022196AA9
:10297000D2020A431A62E0B20021013400F0EEF8FC
:10298000162CF8D11B4B1C005A7852B2002AFBDBE4
:10299000194A5A80194B1A00597EC9090129FBD0DE
:1029A000E421C90099803F21D970537EDB09012BB6
:1029B000FBD0C02300205B011361907000F02EF863
:1029C00063785BB2002BFBDB0D4B0E4A6380D3793F
:1029D000DB09012BFBD04123537010BDFEE7C0463D
:1029E00004000020FFFFFF0010E000E000ED00E029
:1029F00000040040000C00401E4000000040004267
:102A00002140000000480042914202D002D98A1AB7
:102A1000D0407047521A9040FBE70000164A00B5BC
:102A20001300517EC9090129FBD00138042816D8AA
:102A30001969124A0A400F211A615A788A4302F032
:102A4000E3F80308060B0300110001220A435A7041
:102A500000BD11000322F9E711000222F6E7F0237E
:102A600011691B050B430F21136153788B43190028
:102A700002230B435370EBE700400042FFFFFFF0DF
:102A800010B504000E2801D80F34E4B20121200053
:102A900000F0DCF81823102163432B4CE418615636
:102AA000002901D014290DD1284B1800DA79D20958
:102AB000012AFBD002241A78A2431A70C379DB09D9
:102AC000012BFBD022480300427ED209012AFBD011
:102AD0001F2402692140A2430A4302615A7ED2099F
:102AE000012AFBD0022219780A431A705A7ED209B1
:102AF000012AFBD00222197B0A431A731A7ED207DD
:102B0000FCD501221A765A7ED209012AFBD0022274
:102B1000197B0A431A731A7ED207FCD5588B80B2F0
:102B20005A7ED209012AFBD002211A788A431A70F0
:102B30005A7ED209012AFBD0064B1A68064B196847
:102B4000FFF762FF10BDC046F48C00000048004251
:102B5000004000420C00002008000020182330B57F
:102B60001D00040045430820204A5519285601300D
:102B700014D0032912D808006343D156D31802F0A9
:102B800043F802280E1B5868CB010221184A9B18F3
:102B90001A1840321170012282405A6030BD5868C4
:102BA000CB010621124A9B181A18403211700122DB
:102BB00082405A609A61F1E75868CB0106210C4ABD
:102BC0009B181A1840321170012282405A605A61D3
:102BD000E4E75868CB010221054A9B181A184032D5
:102BE0001170012282409A60D8E7C046F48C000040
:102BF000004400411823F0B508245843114A131823
:102C00001C5701341BD0012635005F688356BD4038
:102C10000D4ADB019A18906805420BD10C00601E2A
:102C20008441D2194032107834400336A400B043B6
:102C300020431070044A9B18002901D15D61F0BD4A
:102C40009D61FCE7F48C00000044004118224243DF
:102C5000F8B52C4E0300B218127A52B214000132A9
:102C60000ED0481C00240C280AD801F0CDFF072004
:102C7000202020202020200B0B0B0B00012464427D
:102C80002000F8BD092905D10021D8B2FFF766FF61
:102C90000024F5E70A2902D1D8B20839F6E7002462
:102CA0000B29EDD1D8B20A39FFF758FFE8E7182011
:102CB0004343F2185568F3562C00134ADB016E08A3
:102CC00017389B18C9B204409E19002C0DD00F2450
:102CD00030363278090122401143C9B25B19317094
:102CE00040331A7810431870D2E732000F27303281
:102CF00016785B19BE433143117040331A78104384
:102D00001870BDE7F48C00000044004110B50400C9
:102D1000FFF742FD014B1C6010BDC04610000020B3
:102D20000122024B52421A607047C0461000002038
:102D3000164A10B51368591C26D0013B1360002BAE
:102D400022D172B6124B134A0433934213D9124A5A
:102D500001211000147D0C42FCD02021148BFF3186
:102D60009B085B0021431183D3610C4B138001232B
:102D7000027D1A42FCD0BFF34F8F094B094ADA603B
:102D8000BFF34F8FC046FDE710BDC04610000020C6
:102D900000200000030200000040004102A5FFFFE8
:102DA00000ED00E00400FA050023037101607047A4
:102DB0009446F0B59E1E721E9641624605689207C3
:102DC0002F6836063A4332432A60072505AC24783B
:102DD0000068A4012940214342680024022B00D04E
:102DE0005C03114321434160F0BD30B5C025036849
:102DF000AD031C6812052A402243C0240904A40222
:102E000021401143196003685A6814435C6030BD67
:102E10000123026811680B43136003681A68D20724
:102E2000FCD4DA69D207F9D470470223026811682A
:102E30000B4313600268D3699B07FCD47047026898
:102E4000137E9B0702D40379002BF9D10023037171
:102E50007047002203685A8370470368187E400752
:102E6000C00F70470368187EC0097047802302684E
:102E70005B42117E0B43137670470368588B8007C3
:102E8000C00F704702230268518B0B435383704776
:102E90000368187EC007C00F70470368188DC0B262
:102EA000704703681A7ED207FCD589B219850123C1
:102EB000037118007047012203689A757047012258
:102EC00003681A75704700000368214A30B59342C1
:102ED0002FD0204A93422FD01F4A93422FD01F4A0F
:102EE00093422FD01E4A93422FD01E4A93421FD1A5
:102EF0000E2319220121032599401B48C02401609B
:102F000099082B40AB40FC359D4089000918A4006E
:102F10000859A843C0259D402B0003430B51802333
:102F2000DB011A43114B5A805A7852B2002AFBDB5C
:102F300030BD09231422DDE70A231522DAE70B232B
:102F40001622D7E70C231722D4E70D231822D1E746
:102F500000080042000C0042001000420014004231
:102F600000180042001C004200E100E0000C00409C
:102F7000F8B504000F0016001D00FFF7A5FF2000A4
:102F8000FFF746FF1C21BB000B4071072268090CAC
:102F90000B431360842322689375012F1AD11021EB
:102FA000012E00D008390C4B69431868C00001F0AD
:102FB00035FE0722216802408B895203DB04DB0CBB
:102FC00013438B81226803049089DB0C400B400380
:102FD00018439081F8BDC0460400002000207047CF
:102FE00070B50F26CB1D013902003240D5B22C003E
:102FF00000093034092A00DD07341C70013B8B4284
:10300000F2D170BD10B50C000B4B1868FFF7E8FF4C
:1030100021000A4B08311868FFF7E2FF2100084B36
:1030200010311868FFF7DCFF2100064B18311868D3
:10303000FFF7D6FF202010BD0CA0800040A080002C
:1030400044A0800048A0800008B4024B9C46103881
:1030500008BC604705300000704770473F2070474C
:1030600013B56B460268D971073354681900012201
:10307000A04716BD70B50A260B7892B06E44023395
:1030800005000B703C220021300003F09DFD394803
:1030900001AC069038482421079006202077684626
:1030A000364AA1742281364A364BA281FD3AFF3A54
:1030B0008018C177684623390630C17768460730E3
:1030C000C17702A8C1770720F27703260831694447
:1030D000C87703A9CE7710212B366E4431700926AC
:1030E00021851F3169440E700CA9053E0E703321F5
:1030F0002380022369440B7006360DA90E70224905
:103100003536A1863B216E44307010A86274E27798
:1031100002703D3269446A440B70137040210022F2
:10312000E37023716371A37341336B44218719707A
:103130005A702B7DC039A370A37263770133DBB261
:10314000A3776A7D0B200D0068441543C5773120B5
:10315000684403703A23501C6B44187041230232B8
:103160000A436B441A7021004222084800F0FEFC1A
:1031700012B070BD100104240206052409040000E9
:1031800001020000080B0000070500007405002084
:1031900008B4024B9C46103808BC604775300000EC
:1031A00070B5027D0B790C0000259A420BD10B788B
:1031B0004E78A12B09D1212E05D107221B491C488D
:1031C00000F0D4FC0135280070BD212BFBD1202E4E
:1031D00022D107221549164800F00AFC9622134B0B
:1031E000D200196891421DD1DB79DB071AD4FA208D
:1031F000FFF78CFD00210E4800F0C0FD0125232EB5
:10320000E1D1E378A2781B0213430A4A002108485F
:10321000136000F0B3FDD6E7222EEFD18A78034B7E
:10322000DA71DBE7FFF77CFDE4E7C0461800002019
:10323000740500201400002008B4024B9C4610388E
:1032400008BC6047A131000010B5082200210248E7
:1032500003F0BAFC10BDC0461800002010B5417D37
:10326000006A013100F0FCFA034B1B6801335A1E5F
:103270009341181810BDC0462000002010B5417DB4
:10328000006A023100F002FB10BD10B5417D006AFA
:10329000023100F0C9FA10BD70B50D00417D040087
:1032A000130002312A00006A00F0B6FB002801D1A9
:1032B0000123636070BD000010B5054C23685A1CE3
:1032C00004D103685B69984703002060180010BDB3
:1032D00020000020074A0300106810B5411C03D0ED
:1032E00001235B42136010BD597D186A013100F063
:1032F00043FBF8E72000002010B5FFF7FFF9F423A7
:10330000FF330024984207D9044B0A20DC79631E5E
:103310009C41E4B2FFF728FA200010BD18000020FD
:103320000020704770470000FA239B0010B58360AF
:103330000F4B0022C3820300283383610D4B04002E
:103340004260C2611800503323610830631D21625E
:103350002060DA778323A362813BE36280332363B7
:1033600001F08EFA2100103101F05CFA200010BD4E
:103370000302000054900000022110B5094B1A68A6
:10338000437D5B01D318FF339C7A21439972437DBF
:103390000133DBB25B01D3180122FF33997A0A4370
:1033A0009A7210BD2C0A002010B502490248FFF79E
:1033B000BBFF10BD7405002018050020704710B534
:1033C000040001F009FC200010BD0000F0B58229C6
:1033D00019D1C3B2294D5A01AA189169284C80010C
:1033E0000C40C021890521439161264908334018CA
:1033F0007021506128685B011A5C8A4311003022F9
:103400000A431A54F0BD0029FCD1C026C1B21B4C9E
:103410004B01E3189A681A4DB6052A4032439A6068
:10342000194A800182185A600A0007272468083266
:103430005201115DB9430F000121394311559F69B4
:1034400010493D4040182E439E6158617020115D27
:103450008143080010210143115599680B48A218B7
:10346000084080214903014399609968890B8903C9
:103470009960402311790B431371C3E72C0A002094
:10348000FFFFFF8FA005002060070020FF3F00F036
:10349000EFF3108303600123436072B67047036843
:1034A000002B02D162B6BFF36F8F704773B5836D87
:1034B0000400002B1BD10600A83635786846FFF7BC
:1034C000E7FF019BEDB2013B02D33578EDB2FAE79D
:1034D00068460193FFF7E3FF002D01D1002076BD80
:1034E0002300A4331868A0342368C01AF7E768469D
:1034F000FFF7CEFF22000025019BF432013B02D3EF
:103500001578EDB2FAE768460193FFF7C8FF002D82
:10351000E4D02300F0331868EC34E5E710B5436DD0
:103520004468DBB25A01A218916809480833084080
:10353000802149030143916091685B01890B8903F4
:1035400091602268D318402219790A431A7110BD7C
:10355000FF3F00F0F7B5436D4268DBB2190004008D
:103560000831106849014118C979C90711D55B01B3
:10357000D21893689B049B0C0CD12000FFF7CEFF60
:1035800063681A68636DDBB208335B01D3187F226E
:10359000DA71F7BDE16D002923D12100A4310B6060
:1035A00023000125AC33E56568465360FFF770FFE3
:1035B000260020002100019BA836013BF430F531A4
:1035C0005A1C33D0357002785F1ED2B20A700A7866
:1035D000002A04D120000193FFF7A0FFE8E73B0099
:1035E000EEE72100F0310B600023E3652300603338
:1035F00053606846FFF74CFF01252600200021009C
:10360000019BF436013BA830F5315A1C0ED03570C1
:1036100002785F1ED2B20A700A78002A04D1200014
:103620000193FFF77BFFE8E73B00EEE76846019375
:10363000FFF735FFA4E737B56B46DC1D00230D000F
:10364000237001F01DF9210001F0A9F82B6818186A
:10365000286020783EBD00000078002810D00121AD
:10366000084B1B681A898A431A810822198B0A435E
:103670001A830422198B0A431A830022024B1A6010
:103680007047C0462C0A0020240A002010B50F4ABB
:1036900093699B0B9B03936113680222FF331A7299
:1036A0009879823A02439A711A7A9207FCD57F245C
:1036B000074A2140937A0800A3431900802301435D
:1036C0009172917A5B420B43937210BD2C0A0020D9
:1036D0000050004110B50C0001F0D2F8210001F0BB
:1036E00091F8002804D1034A93699B0B9B039361D3
:1036F00010BDC0462C0A0020F8B50D00832A19D150
:10370000CBB23B4C5A01A21891693A48AD0108402E
:10371000C021890501439161374920686D187021E6
:10372000083355615B011A5C8A43110040220A4349
:103730001A54F8BD022A55D1304A8B0098580028F7
:1037400002D003685B699847F82001F041FA040051
:10375000274E2B4B4660036040220021083003F0C7
:1037600033FA22000023A032A3646565E364236575
:10377000A365E3655360D3641372136013654C3221
:1037800013725372FF222B0013405901711888687D
:10379000184F08330740C0208005384388603068E0
:1037A00007265B01195CAD00B1430E0003213143D4
:1037B00019542300616D606811404901411860335C
:1037C0004B60616D63680A401B6852019B180122BF
:1037D000FF33997A20000A439A72FFF79FFE074B46
:1037E0005C51A6E711002800FFF7F0FDA1E7C046F5
:1037F0002C0A0020FFFFFF8FA00500207805002085
:10380000BC90000070B505000124064BA200D25800
:10381000002A06D0210028000134FFF76DFF0A2C92
:10382000F3D170BD4C0500200B4BCAB20B48890187
:10383000C9185301C318596199690832890B890362
:103840009961036852019A180223D3715179823B1E
:103850000B4353717047C046A00500202C0A00207E
:10386000084B8A00D05810B5002803D003689B6825
:10387000984710BDC9B2044B4901591888688004A3
:10388000800CF6E7780500202C0A002010B50C000B
:10389000FFF7E6FF00280CD0064BE4B21B680834A3
:1038A00064011C19802362795B4213436371022314
:1038B000E37110BD2C0A0020F0B51C002A4B85B026
:1038C0001B6807000D000292002B4AD0274B8A008C
:1038D000D058002808D0036822005B6802999847F6
:1038E0000400200005B0F0BD3800FFF7B9FF8442A6
:1038F00004D929003800FFF7B3FF04000121EBB21F
:103900001B4E03935B010193F21893689B0B9B037F
:103910009360019A336802989B18FF335A7A0A43DE
:103920005A72144BA901C918220003F031F9002C76
:10393000D7D029003800FFF793FF0028D1D14021CC
:10394000039B326808335B01D3181879014319715E
:103950000121D971019BD318FF339A7A0A439A72D5
:10396000BFE701246442BCE7240A00207805002058
:103970002C0A00206007002013B56B46DC1D2200D6
:103980000123FFF799FF012801D1207816BD0120FE
:103990004042FBE770B5CBB2124A13485C01890183
:1039A0008918021951609168104D08330D4080212B
:1039B00049032943402591609168890B89039160EF
:1039C00001685A018A1816793543157195796D0683
:1039D000FCD55B01C918CB79DB07FCD500198068E1
:1039E000C0B270BD600700202C0A0020FF3F00F02D
:1039F00070B50D0000211400FFF7CCFFA04200D9E4
:103A0000200000230349A34203D0CA5CEA540133D7
:103A1000F9E770BD60070020F0B51E003A4B85B095
:103A20001B680F000192002B35D08023DB019E42E2
:103A300031D80025354B8A01D3180293002E2CD0A3
:103A4000334B1B680393FF233B401C000093083457
:103A5000039B64011C19A379DB0921D02D4B2E494E
:103A6000186801F0DBF82D4B1721584301F0D6F808
:103A70002B4BE279920713D4DA5D002A01D1013889
:103A8000F7D20122DA55009B5A01214B9B189A6903
:103A9000920B92039A6101256D42280005B0F0BD9A
:103AA00000221F4B3400DA553F2E09D9009B4024D9
:103AB0005A01174B9B188022996912060A439A6192
:103AC00022000199029803F063F8009BA1045A01B7
:103AD0000F4B890C9B18029A2D195A619A69361B53
:103AE000920B92030A439A61009B039A08335B018D
:103AF000D3180222DA715979823A0A435A71019B2A
:103B00001B1901939AE7C046240A0020A005002053
:103B10002C0A00200400002040420F007011010018
:103B20009505002070B50D001C000D4BAE01F61878
:103B300011003000220003F02BF8EDB209496D01AD
:103B40004D196E61AB69084A20001340AB61AB6947
:103B5000A2049B0B920C9B031343AB6170BDC04648
:103B6000A00500202C0A0020FF3F00F0F7B5104B05
:103B700001901B780F001500002B0CD10D4B160087
:103B80001C78002C09D00C4E0C483488201864197D
:103B900002F0FEFF34802800FEBD002EFBD03A1953
:103BA000330000210198FFF7BDFF2418361AF4E70F
:103BB00020090020210A0020220A002021090020DB
:103BC000F8B50F0016000024012A26D9100002F0D3
:103BD000B9FF0500380003F041FD03230222013044
:103BE000400028706B7096420DD9397800290AD0B0
:103BF000531CDBB20137A9549E4203D00232EC546D
:103C0000D2B2F0E7320029000548FFF7AFFF441EAB
:103C1000A041C4B2280002F09FFF2000F8BDC046BA
:103C200074050020F0B50024012685B0184B0F0064
:103C300069461E7005000094FFF7FDFC154B01A9B5
:103C40000B806A3BFF3BCB715A330B72009B8C712C
:103C500009334B800E4B4E7108711C703A00092FCE
:103C60000FD00D4F09223E700C4E28000094348076
:103C7000FFF77CFF69462800FFF7DDFC3288084922
:103C80003C702800FFF772FF012005B0F0BDC04670
:103C90002009002009020000210A0020220A002039
:103CA0002109002070B5CE7892B005000C00022EDC
:103CB0000BD18B79C9792C4809021943FFF7B2FF60
:103CC000411E8841C0B212B070BD00F0D9FD210084
:103CD00000F079FD002803D0C117081AC00FF2E7E1
:103CE000012E0ED1E279A37912021A431F49112A3B
:103CF00013D8D2B2002A10D02800FFF737FF0120D6
:103D0000E1E7032EDFD1A378002B08D1E279A37974
:103D100012021A431649032AEBD90A78ECE7022B60
:103D200008D1E279A379120212491A432800FFF759
:103D300047FFC8E7012B05D1E279A37912021A43A4
:103D40000D49F3E7032BBED14122010001A802F087
:103D50003BFF00F095FD01A900F045FDE279A37954
:103D600012021A4301A9E1E774050020F89000004F
:103D7000E8900000D8900000EC900000CBB204491D
:103D80005B01C9188B699B0B9B038B617047C04615
:103D90002C0A002037B5050048780C000B2810D8F5
:103DA00000F032FF061B0F2B0F404561494C5A5D56
:103DB000097801AA002906D1022311802800FFF703
:103DC000B1FE01203EBD00231380284B1B78012B40
:103DD00000D1137002230021F0E78A780023012A22
:103DE00003D101AA1380224BF0E7204A1370214A25
:103DF00093699B0B9B039361E3E78C78012C06D1BD
:103E000000211B4B01AA1C7011702300D6E7012072
:103E1000002CD7D1154B174A187093699B0B9B0345
:103E20009361CFE789782800FFF730FCC9E72800C5
:103E3000FFF738FFC6E701230F4ACCE70B780020D5
:103E4000DB06BFD12800FFF7DDFCA2780A4B0B4848
:103E50001A60FFF791FACAE70123094ABBE78A789B
:103E6000074B1A60C3E70020ACE7C046940500206A
:103E70009C0500202C0A0020240A002018050020A0
:103E8000280A00203A4BF7B51E780500002E5FD1B6
:103E9000384C23689A8B12070DD5082231009A837B
:103EA0003000FFF793FA10222368FF33997A0A4310
:103EB0009A72314B1E6023689A8B520701D50422F7
:103EC0009A83FF331A7A920603D52022597A0A433D
:103ED0005A721A7AD20623D569460800274AC0CA00
:103EE000C0C0A268920B9203A2604022587902439C
:103EF0005A7160230A7828001A422AD1FFF74AFF34
:103F00002368FF33002827D08022997952420A4340
:103F10009A711A7A520603D54022597A0A435A7284
:103F20007F2601252368FF331E722F002368083780
:103F30007F01DB19DB79002B07D0114BAA00D05889
:103F400000280DD003681B6898470135082DECD177
:103F5000F7BDFFF7BFFBD3E720210A4A9171D8E7ED
:103F600029000948FFF7DEF92368DF19FE71ECE745
:103F7000210A00202C0A0020240A002060070020CB
:103F800078050020FF5000411805002010B50248B8
:103F9000FFF778FF10BDC0467405002080235B004A
:103FA0000380002343600733037270478300014896
:103FB000C01870474C050020836C402B09D03F226D
:103FC000036CC154036C013313400364836C0133ED
:103FD00083647047F7B505006846FFF759FA002675
:103FE0004022019B013B02D32E6D961BFAE76846E7
:103FF0000193FFF754FAAB6D6846002B4FD1FFF7E2
:1040000047FA2900019BA831013B5A1C0CD00C78BF
:104010005A1EE4B2002C05D168460193FFF73FFA1F
:104020002000FEBD1300F0E7684601930024FFF76F
:1040300036FA2A002900A0321368A431B4420ED007
:10404000086898420BD92800591CEB18116060339E
:1040500019780830C9B2FFF7AFFF0134E9E7096802
:104060009942DDD1002313600133AB656846FFF749
:104070000FFA2F002A000021019BA837013BF532DF
:10408000581CC9D0397010785E1E002805D01170F8
:1040900028000193FFF742FAEBE73300F0E7FFF760
:1040A000F7F92900019BF431013B5A1C06D00C782A
:1040B0005A1EE4B2002CAFD01300F6E76846019315
:1040C0000024FFF7ECF92A002900EC321368F031E4
:1040D000B44202D0086898421DD8096899429FD11D
:1040E000002368461360AB65FFF7D2F92F002A0062
:1040F0000021019BF437013BF532581C00D18BE7BE
:10410000397010785E1E002811D0117028000193BC
:10411000FFF704FAEAE72800591CEB181160AC33EA
:1041200019780830C9B2FFF747FF0134CBE73300F5
:10413000E3E710B50400FFF74DFF206D10BD10B58B
:104140000400FFF747FF236D002B03D0E36CE41856
:10415000207A10BD01204042FBE7F7B517000E00A2
:104160000400FFF737FF6846FFF792F93F2200256A
:104170009446019B013B5A1C19D0BD4215D2226DB9
:10418000002A12D00121226D4942002A0AD060463D
:10419000E26CA218117AE26C01320240E264226DF4
:1041A000013A226571550135E7E7013BE3E76846CF
:1041B0000193FFF774F92800FEBD0000014B024A8D
:1041C0001A6070472C0A0020005000412023F7B5E8
:1041D000474A0500D1690F200B43D36101224549AD
:1041E0000B7813430B70444B1978814319700621E7
:1041F0001C782143197041490C7822430A701A78BF
:1042000002401A70602219780A431A703C4B3D4AEA
:104210005A805F78FF09FCD13B48FEF769FA012319
:104220003A4C3B4E2268300011780B4313708022C9
:104230003900520002F0C8FC22689378DB07FCD4F6
:1042400056621F26334B1B68590B980C9B0131405B
:1042500030405B0FB14200D105211F2800D1023848
:10426000072B00D1043B31408901178D01912A4968
:1042700030400F40019939431185118D0700B1433A
:10428000080038431085118D1803244B7F260B40FE
:1042900003430C2013850823D17881430B4303216A
:1042A000D3702268D3788B4301390B43D3702268D3
:1042B0001378334013700423226816783343137045
:1042C0002268C1241389A40083431548138103592C
:1042D0001B021B0A03518023036013781148194302
:1042E000012311702B700021FEF7B6FEF7BDC0460A
:1042F00000040040584400413C44004159440041FE
:10430000000C0040064000008D3F00002C0A0020F9
:10431000300A0020246080003FF8FFFFFF8FFFFF7E
:1043200000E100E0180500200120704710B5036887
:10433000014A1B6A984710BD13040000FC30006A54
:10434000704787239B00C018C36880204000C01AB4
:1043500070470300FC331A6A002A03D0DB69C018D7
:10436000007D704701204042FBE710B50400006962
:10437000FEF74EFD22000023FC329361D3611362ED
:1043800087229200A4186360A360E36010BD8723B6
:1043900010B59B00C218D368002BFCD10069FEF752
:1043A0004EFD10BDF0200140303948424841704771
:1043B000F0231B011940802306209B0099420AD05C
:1043C0000133FF330130994205D0802302385B006E
:1043D000994200D0002070470F20014000200129A1
:1043E00003D00239481E8141481C70478B23F0B529
:1043F000182685B002919B000400C05C33000821A0
:104400004343324D1700EB185956FEF71FFC304B53
:104410000821E05C33004343EB185956FEF716FCC5
:104420002C4BE25C0393022A09D11133E05CFF2894
:1044300005D008214643AE197156FEF707FC8C26BD
:10444000B600A05DFF2819D00121FEF787FB1822D6
:10445000A35D21495A43AB56AD18DB0158188D2195
:10446000890060501D4901225B188E21890063502C
:1044700069688A408F21890062501A600122029B7C
:1044800011002069FEF774FD39002000FFF790FF4E
:10449000390005002000FFF79FFF390006002000CB
:1044A000FFF780FF33000090290020690122FEF70A
:1044B0007FFC0B4B2069E25C039BE15CFEF795FC03
:1044C0002069FEF7B2FC05B0F0BDC046F48C0000D8
:1044D0002D0200002F020000184400411444004146
:1044E0002E020000802210B504005200002102F0CC
:1044F0006BFB23000022FC335A6020009A60DA60D4
:1045000010BD0000F7B51D0008AB1B780400009338
:1045100009AB1B781600019300234360FA239B002C
:104520008360114B0F00083303601430FFF7DAFF8C
:1045300020002130FF30FFF7D5FF8B236A469B0018
:104540002761E654094B1278E554094B2000E254E8
:104550006A46084B1279E2548C22313BFF3B9200B1
:10456000A3541032A354FEBD0C9100002D02000094
:104570002E0200002F020000F7B5EFF31083009326
:104580000123019372B680260200FF25019BFC32B5
:104590007600013B5C1C0FD0D4685F1EB44209D08A
:1045A00054680155546801342C405460D468013477
:1045B000D460EEE73B00EDE768460193FEF76FFF3E
:1045C000F7BD13B5EFF3108300930123019372B687
:1045D000019B5A1E0192002B15D00300FC33DA68B0
:1045E000002A0DD09A68845C9A680132D2B29A602F
:1045F000DA68013ADA606846FEF751FF200016BD1E
:1046000001246442F7E701246846FEF748FF64424C
:10461000F4E710B504000069FEF72FFC002805D070
:104620002069FEF73AFC2069FEF72CFC2069FEF7B2
:1046300014FC00281BD02069FEF72FFC010020008D
:104640001430FFF799FF8C239B00E35CFF2B0ED007
:104650002300FC331A6A80235B009B1A092B06DCBB
:104660008D238F229B009200E358A2581A60206984
:10467000FEF70EFC00280ED087239B00E318DB68B2
:10468000002B14D020002130FF30FFF79AFFC1B279
:104690002069FEF706FC2069FEF7E4FB002805D040
:1046A0002069FEF7E3FB2069FEF7D3FB10BD20690C
:1046B000FEF705FCEFE70000F8B5040000690D0007
:1046C000FEF7E6FB87239B00E618002802D0F3687C
:1046D000002B34D001278022F3685200934223D16B
:1046E000EFF310833B4210D1174B5B68DB05DB0D0A
:1046F000F1D0103B5BB2002B10DAF13A1340083BCB
:104700009B08124A9B009B181B682069FEF7C0FBA0
:104710000028E0D02000FFF77CFFDCE79B08C033D7
:104720000B4A9B009B58F0E720002130FF30290006
:10473000FFF722FF2069FEF7BEFB0120F8BD29002C
:104740002069FEF7AEFBF8E700ED00E01CED00E0AD
:1047500000E100E010B504001430FFF732FF8C23B5
:104760009B00E35CFF2B0ED02300FC331A6A8023EE
:104770005B009B1A0A2B06DD8E238F229B00920082
:10478000E358A2581A6010BD10B51C00431A0298D5
:10479000511A001B584300F0CBFA001910BD70B538
:1047A0000E0000254468002C0BD0236831005B68A4
:1047B00020009847002802DB2D18E468F3E7012564
:1047C0006D42280070BD70B50D004468002C08D003
:1047D000236829009B6820009847002802D1E468DC
:1047E000F4E7200070BD70B50D004468002C07D0C0
:1047F000236829002000DB689847E4682D18F5E756
:104800002C7070BD70B50D004468002C08D0236872
:1048100029001B6820009847002802D1E468F4E7CB
:10482000200070BDF8B542788B790D00017A9B1895
:10483000040000208B4222DC6368834219D165604A
:10484000002623786A71EA792B719B182370AB7963
:10485000B34213D9AB68B7006078DF19FFF7A6FB46
:104860003B68013603606378F6B201336370EEE7AC
:104870000B00D9680029FBD1DD60E1E70120F8BD1C
:1048800070B50126054D064C2B68334203D120003C
:10489000FFF784FB2E60200070BDC046300B002067
:1048A000340B0020F7B506000D000C008B180193A7
:1048B000019B671B9C4207D0336821781B6830003E
:1048C000984701340028F3D13800FEBD70B50400CC
:1048D00008000D0002F0C2FE2368020029005B6898
:1048E0002000984770BD10B50B1E02D0FFF7EEFFF9
:1048F0000300180010BD10B503688A685B6809687A
:10490000984710BD10B5FFF7EEFF10BD10B5036856
:104910001B68984710BD000010B50249FFF7D6FF8D
:1049200010BDC0464091000070B50500FFF7E3FFE1
:1049300004002800FFF7F0FF201870BDF0B58BB021
:104940006B461500002205330600DA770800012DBA
:1049500000D80A2509AC290000F0E6F9CAB2130014
:1049600037330700DBB2092902D813003033DBB23A
:10497000013C2370002FEED121003000FFF7B3FF80
:104980000BB0F0BDF8B506000C00151E04D103688D
:10499000C9B21B689847F8BD0A2A0CD100290BDA66
:1049A0002D21FFF7B3FF614207002A003000FFF717
:1049B000C5FF3818EFE7D2B221003000FFF7BEFF85
:1049C000E9E710B5FFF7DEFF10BD10B50400006881
:1049D000002801D002F0C0F8200010BD10B504007E
:1049E0000068002801D002F0B7F800232360A3601C
:1049F000636010BD70B504000D000068013102F065
:104A0000F1FD031E01D0012028C470BD036810B55C
:104A10000400002B04D043688B4201D3012010BD59
:104A20002000FFF7E7FF0028F9D0A368002BF5D19D
:104A300022681370F2E770B50E0011000400150033
:104A4000FFF7E4FF002804D12000FFF7C7FF200094
:104A500070BD2A003100A560206802F099F800239B
:104A60002268A1685354F2E770B5050008000C00F5
:104A700002F0F4FD210002002800FFF7DCFF70BD0A
:104A800010B50B000400884205D00968002904D045
:104A90009A68FFF7D0FF200010BDFFF79FFFFAE7ED
:104AA000002310B50400036043608360FFF7E8FF54
:104AB000200010BD10B50400002903D0FFF7D4FF7B
:104AC000200010BDFFF78AFFFAE730B5D5B0190016
:104AD00058AB040010001A78002323606360A360C1
:104AE000131C0A2A00D90A23DBB29A1C03AD52B266
:104AF000009500F075F801002000FFF7DBFF2000B3
:104B000055B030BDF7B504000F001600002903D1E1
:104B1000002301930198FEBD01230193002AF9D0DF
:104B20008368D5182900FFF771FF0028F0D02368AB
:104B3000A26839009818320002F02AF8002223688F
:104B4000A5605A55E6E770B5050008000C0002F0B4
:104B500085FD210002002800FFF7D4FF70BD00236F
:104B600010B5994202D0FFF7EEFF0300180010BD08
:104B700010B50400002904D12000FFF72FFF20000A
:104B800010BDFFF7ECFF0028F6D0F8E770470000F3
:104B900010B5FDF7C1FE01F0B1FFFFF7F7FF0120EF
:104BA000FDF7E2FD084C2000FFF710FB2000FEF7A8
:104BB00053FDFDF755FBFDF7F5FA044B002BFAD03A
:104BC00000E000BFF7E7C0467405002000000000C9
:104BD00010B501F0B7FF10BD10B501F0BDFF10BD5D
:104BE00030B5040087B00D00064901A802F016FD9B
:104BF00022002B0001A90A9802F010FD0A9807B0C4
:104C000030BDC0464391000002B4714649084900D6
:104C1000095C49008E4402BC7047C046002243082C
:104C20008B4274D303098B425FD3030A8B4244D374
:104C3000030B8B4228D3030C8B420DD3FF220902B6
:104C400012BA030C8B4202D31212090265D0030B75
:104C50008B4219D300E0090AC30B8B4201D3CB036B
:104C6000C01A5241830B8B4201D38B03C01A5241AD
:104C7000430B8B4201D34B03C01A5241030B8B42AF
:104C800001D30B03C01A5241C30A8B4201D3CB029A
:104C9000C01A5241830A8B4201D38B02C01A52417F
:104CA000430A8B4201D34B02C01A5241030A8B4282
:104CB00001D30B02C01A5241CDD2C3098B4201D39A
:104CC000CB01C01A524183098B4201D38B01C01A18
:104CD000524143098B4201D34B01C01A524103098F
:104CE0008B4201D30B01C01A5241C3088B4201D33E
:104CF000CB00C01A524183088B4201D38B00C01AEB
:104D0000524143088B4201D34B00C01A5241411A11
:104D100000D20146524110467047FFE701B500201E
:104D200000F0F0F802BDC0460029F7D076E77047E2
:104D300003460B437FD4002243088B4274D30309FC
:104D40008B425FD3030A8B4244D3030B8B4228D39D
:104D5000030C8B420DD3FF22090212BA030C8B42C3
:104D600002D31212090265D0030B8B4219D300E063
:104D7000090AC30B8B4201D3CB03C01A5241830BE8
:104D80008B4201D38B03C01A5241430B8B4201D398
:104D90004B03C01A5241030B8B4201D30B03C01AC1
:104DA0005241C30A8B4201D3CB02C01A5241830A3B
:104DB0008B4201D38B02C01A5241430A8B4201D36A
:104DC0004B02C01A5241030A8B4201D30B02C01A94
:104DD0005241CDD2C3098B4201D3CB01C01A5241FB
:104DE00083098B4201D38B01C01A524143098B4284
:104DF00001D34B01C01A524103098B4201D30B016D
:104E0000C01A5241C3088B4201D3CB00C01A524191
:104E100083088B4201D38B00C01A524143088B4256
:104E200001D34B00C01A5241411A00D201465241EF
:104E3000104670475DE0CA0F00D04942031000D30E
:104E40004042534000229C4603098B422DD3030A63
:104E50008B4212D3FC22890112BA030A8B420CD373
:104E6000890192118B4208D3890192118B4204D39C
:104E700089013AD0921100E08909C3098B4201D31C
:104E8000CB01C01A524183098B4201D38B01C01A56
:104E9000524143098B4201D34B01C01A52410309CD
:104EA0008B4201D30B01C01A5241C3088B4201D37C
:104EB000CB00C01A524183088B4201D38B00C01A29
:104EC0005241D9D243088B4201D34B00C01A524100
:104ED000411A00D20146634652415B10104601D38D
:104EE0004042002B00D54942704763465B1000D317
:104EF000404201B5002000F005F802BD0029F8D0BD
:104F000016E770477047C0468446101C62468C46C0
:104F1000191C634600E0C0461FB500F0F1FE0028F2
:104F200001D40021C8421FBD10B500F049FE404227
:104F3000013010BD10B500F0E3FE002801DB0020B9
:104F400010BD012010BDC04610B500F0D9FE0028EC
:104F500001DD002010BD012010BDC04610B500F0DD
:104F60006BFE002801DC002010BD012010BDC046F2
:104F700010B500F061FE002801DA002010BD01200C
:104F800010BDC046F0B54F464646D6460C00090354
:104F9000C0B5490A470F5E0039431F03DB0F9C462B
:104FA00065007B0A570F1F436D0DE40F760DA14678
:104FB000C000B846D200AB1B64457BD0002B5FDD40
:104FC000002E00D0A4E03E00164300D112E15E1E88
:104FD000002E00D09EE1871A4346B8428041012549
:104FE000C91A4042091A0B0200D431E149024E0AA3
:104FF000002E00D16EE1300001F062FD0300083B9D
:105000001F2B00DD61E120223900D21A9E40D140E1
:105010009F400E439D4200DD51E15D1B6B1C1F2B29
:1050200000DD7CE12021C91A3D0030008F4088401E
:10503000DD40791E8F41310007222843D9400025E9
:1050400007433A40002A09D00F233B40042B05D0E8
:105050003B1DBB42BF417F42C9191F000B0200D458
:1050600026E26A1CC64B55056D0D9A4200D106E139
:10507000C44AFF080A40530752023B43120B8EE01A
:10508000002B00D0B8E06B1C5B055B0D012B00DC36
:1050900030E1871A4346B842B641CB1A76429E1B8E
:1050A000330200D54CE13B003343A1D10022002460
:1050B000002570E0002B00DCE5E0002E00D183E04D
:1050C000AF4EB54260D0802636043743B846382B01
:1050D00000DC3EE1434613431F007A1E97413F1810
:1050E00087428041404209180B0200D4B0E0A44B33
:1050F00001359D4200D1C3E0A24A7B080A4001214C
:105100000F401F435108D30707221F433A4099E736
:105110009B4EB54238D0802636043743B846382BEC
:1051200000DDDCE01F2B00DC30E11E004746203EA6
:10513000F740BC46202B04D04026F31A46469E403A
:105140003243170063467A1E97411F43CCE0002B81
:1051500000D104E24346134300D159E14B07C00894
:1051600018438023C9081B03194208D04546ED089F
:105170001D4204D14346D008590708432900420F75
:10518000C9007F4D1143C0004B07CA087C49C008C5
:1051900003438D4268D012036D05120B6D0D002183
:1051A00012031800130B0A0D12051A43764B2D0536
:1051B00013402B435B00E4075B08234319001CBC2E
:1051C00090469946A246F0BD3E00164312D05E1EA0
:1051D000002E00D000E187188742804141444042C0
:1051E000091801250B0233D5022585E764463300F3
:1051F000414610001D00C7E7002D00D0DAE00C008A
:105200000443F3D05C1C00D19FE15D4CA64200D169
:105210002FE1DB43382B00DD66E11F2B00DD83E14E
:1052200020240500E41A0F00DD40D940A040434689
:10523000A7405B1A441EA04198462F433843171AD3
:10524000BA42924143465242991A64463500CAE630
:1052500007223A40002A00D0F6E64B07CA08484920
:10526000FF083B438D4296D11900114300D19EE1C6
:10527000802109030A431203120B414D8FE71500E9
:10528000002200238BE7002B00D0C7E06B1C5F05DA
:105290007F0D012F00DCF1E0394DAB4200D1B9E0C8
:1052A00085180A0085428941424449425118072223
:1052B000CF076D082F4349083A401D00C2E6072278
:1052C0003049ED1A31403A40BCE63E00283886406D
:1052D00000279FE6380001F0F3FB20308EE64346BE
:1052E00013431F007A1E9741C71BB84280414042BA
:1052F000091A78E60E003B0006431343002D61D1E6
:10530000002E00D0F4E0002B00D11BE164463900F0
:10531000100039E71A4FBB427AD03300FFE6300065
:105320001F3DE840202B03D04021CB1A9E4037433D
:105330007B1E9F41072207433A400021002589E751
:10534000171A4346BA42B641591A76428E1B644632
:105350004EE61F2B00DDADE020264746F61AB7408B
:10536000B9461700B246DF404E463E433700564628
:10537000B240561EB24117434246DA408918AEE6A3
:10538000FF070000FFFF7FFFFFFF0F80202647463B
:10539000F61AB740B9461700B246DF404E463E43C4
:1053A00037005646B240561EB24117434246DA40D5
:1053B000891A99E77F4CA6425BD0802424045B4283
:1053C000214327E7002E0CD1002B00D1CBE064460F
:1053D00039001000774DD7E6764FBB4218D0330026
:1053E00075E6002B14D04B07C00818438023C9086A
:1053F0001B03194207D0FC081C4204D17907D008CE
:105400000843E14621004C46420FC9001143C00049
:10541000684DB9E61D0000220023C0E6002D5BD1D7
:105420000D00054300D1E2E65D1C00D1B0E0614D06
:10543000AE421FD0DB43382B71DC1F2B00DD96E022
:1054400020250F00ED1AAF40B9460700AA46DF40FD
:105450004D463D432F005546A840D940451EA84122
:1054600088440743BF189742924151424144350056
:105470003AE6644635004146100085E60B000343DA
:10548000002D00D063E6002BF5D04346134300D136
:105490007AE6871887428041072241444042091832
:1054A0003A400B0200D4D5E6434B01351940C9E51B
:1054B000380069E61E004746203EF740BC46202BD8
:1054C00004D04026F31A46469E40324317006346F6
:1054D0007A1E97411F4302E6364DAE42CAD0802560
:1054E0002D045B422943A6E70843411E8841A6E6F6
:1054F000002B00D148E6871A4346B842B641CB1A82
:1055000076429E1B33024BD5171A4346BA4292414C
:10551000591A5242891A072264463A4092E50143D9
:105520000F00791E8F419DE71C000F00203CE740D3
:10553000202B03D04024E31A99400843411E8841A0
:1055400038437CE60022002425E6171A4346BA4277
:105550009241591A5242891A6446350043E5414640
:105560001000144D10E680220024120380E61D0076
:105570000F00203DEF40BC46202B03D04025EB1A06
:105580009940084307006346781E87411F4369E737
:10559000871897429B4141445B42C9183500A3E5F7
:1055A0003B003343CED0072231003A4052E600237D
:1055B0001A00F4E5FF070000FFFF7FFFF0B5574634
:1055C000DE464E464546E0B5834607000E034800DA
:1055D00085B092461C00360B400DCD0F002800D13F
:1055E0009DE0954B984239D08023F6001B041E4362
:1055F000924A7B0F334399469446030063440093D9
:1056000000230026FF00029323031B0B9846630030
:10561000E40F52465B0D019400D1B3E086498B4202
:1056200000D19EE04246D100802212040A43514636
:10563000490F11438B46814952468C460099634479
:10564000CB1A0021D20000932B0063409A460F2E04
:1056500000D905E17A4BB6009B599F465B46334320
:10566000994600D0B8E00223082600270090029354
:10567000CAE7CB463A0002990195019B9A46022956
:1056800027D0032900D180E2012944D06D49009B35
:105690008C4663441C00002C38DD530700D013E215
:1056A000D2085B46DB0109D55946674B19408B464A
:1056B0008021C9008C46009B63441C00634B9C42C4
:1056C00007DC5B4664055F075B0217431B0B620D3B
:1056D00002E000230027584A00211B031C0B0B0D7E
:1056E0001B05234314055A4A380013401C435346F4
:1056F0006400DB0764081C43210005B03CBC9046F5
:105700009946A246AB46F0BD0122524201231B1B23
:10571000382B00DCADE1002200230027DCE75B46EC
:10572000334399465ED0002E00D18AE1300001F06B
:10573000C7F903000B3B1C2B00DD7BE11D22D31AB4
:105740005A460100DA4008398E4013005F46334361
:1057500099468F403F4B00261B1A0093002302936B
:1057600052E7414653460B433B499B468C46009BC0
:10577000634400935B46002B3BD1022300221E436F
:10578000022161E7434613439B4637D04346002B33
:1057900000D162E1404601F093F903000B3B1C2B62
:1057A00000DD53E102004146083A914088461D2140
:1057B000CB1A5146D9400B0041460B439B465346FA
:1057C00093401A00009B25499C46604403008C4688
:1057D00063440093002137E70323B14600900C2671
:1057E000029311E70023009301330426002702935C
:1057F0000AE70323C3461E43032125E701331E4363
:105800000022012120E700239A46802300271B0362
:10581000094A61E7802349461B03194200D1E2E0AF
:105820005946194200D0DEE00B431B0317001B0B47
:10583000A246014A50E7C046FF07000001FCFFFFF7
:105840004C910000FF030000FFFFFFFEFE07000079
:10585000FFFF0F800DFCFFFF01F8FFFFF3030000C7
:10586000D94500D9CBE000D1C6E03C00484600272E
:10587000009B013B00935B46160E1B021E43130266
:10588000984633041B0C9946310C0191FFF74CFAF2
:105890004A4642430B04210C050019438A4207D9AA
:1058A0008919013D8E4203D88A4201D9851E891982
:1058B000881A0199FFF738FA09048C464A462104F0
:1058C00064464243090C030021438A4204D98919E2
:1058D000013B8E4200D8F1E02D041D43AB46434608
:1058E000891A4246280C12041D0C5B46140C220037
:1058F0001B041B0C5A4303946B43444302956843B7
:105900001B19150CEB189C4203D980246402A44691
:1059100060441C0C15041B042D0C20185D198142D9
:1059200077D373D00C1AA24A7D1BAF42BF41944675
:10593000009B7F426344E01B1C00864200D1DBE0F9
:105940000199FFF7F1F94A4642430B04290C07007D
:1059500019438A4207D98919013F8E4203D88A42E6
:1059600001D9871E8919881A0199FFF7DDF9090401
:105970004A46894629044D464243090C03002943FF
:105980008A4207D98919013B8E4203D88A4201D93C
:10599000831E89193F04891A3A00039F1A4338006D
:1059A00013041B0C584381460298150C6F43434364
:1059B00045434846000C8446DB1963449F4203D9A3
:1059C000802040028446654448461F0C00041B04A6
:1059D000000C7D191818A94200D284E000D17FE0A4
:1059E00001231A4357E680234A461B0313431B0334
:1059F0001B0BAA466F4A6FE6BA4200D935E74B4601
:105A0000DC0758087B081C43FF0734E70024AF423B
:105A100089D247444745A4415B466442A4196418AF
:105A2000013BA6421ED2A0426DD800D1B6E0241A96
:105A30009B4678E703005A46283B9A400027914648
:105A400088E6584601F03CF8203072E603005246E2
:105A5000283B9A4093460022B4E6504601F030F8C5
:105A600020309AE6A642E2D1B845DCD9341A9B46EA
:105A700059E71F2B65DC504C0099A4465C466144F5
:105A800008008C4011008240D940501E82410C43D6
:105A900014435A46DA401300620709D00F2222400D
:105AA000042A05D02200141D9442894149425B1802
:105AB0001A0262D50122002300270DE68A4200D88F
:105AC0000AE7831E891907E70F231340042B00D12F
:105AD000E6E5171D9742924153429B44FA08E0E5E0
:105AE000002800D1D7E57118531EB14227D3A9422F
:105AF00015D358D01A0073E7002B00DC04E601230D
:105B000000229B44CDE502234744474589415B423F
:105B10009C46494289190C19E344241A03E7434679
:105B20005F0047459B41B8465B429E19023A89197E
:105B3000A94200D054E7404500D051E7ABE51A0038
:105B4000F6E71F215F4649420C1BE740202B07D098
:105B50001A49009B8C46634418005B4683401A43F5
:105B6000501E82413A4307270023174009D00F21D6
:105B7000002311401400042995D122005F075B0225
:105B80001B0BD20817430022A6E5802359461B03AE
:105B90000B431B0317001B0B064A9DE5BD42B2D801
:105BA0009B460024BFE68045B9D31A00C3E7C04630
:105BB000FF030000FF0700001E0400003E04000079
:105BC000F0B54F464646D6468446C0B58046194E87
:105BD00018030F034D00000B5C0082463F0B6D0D58
:105BE000C90F9146640DDB0F0120B5420AD0B442C3
:105BF00003D0A54201D157450CD01CBC9046994614
:105C0000A246F0BD66463E43F7D1AC42F5D15446BC
:105C10001443F2D10120C845EFD1994207D0002D9D
:105C2000EBD163461F433800471EB841E5E700202B
:105C3000E3E7C046FF070000F0B54F464646D646AC
:105C40004D00C0B50E03C90F8A462C491F035C00E6
:105C50008046360B6D0D91463F0B640DDB0F8D4278
:105C60001ED08C4216D0002D1ED130438446002C0D
:105C700001D13A4323D06246002A1AD09A4529D04E
:105C8000514602200139084001381CBC9046994613
:105C9000A246F0BD39001143E5D002204042F4E7AE
:105CA0003043FAD1AC420FD0002C0FD13A43E7D0A9
:105CB0000CE00122013B934318000130E5E7634605
:105CC0000020002BE1D0DBE73A43E6D19A45D7D15B
:105CD000A542D5DCA54205DBBE42D1D808D00020C4
:105CE000BE42D2D250460123013898430130CCE75E
:105CF000C845C5D80020C845F4D3C6E7FF07000053
:105D0000F0B54F464646D6464D00C0B50E03C90F06
:105D10008A462E491F035C008046360B6D0D914666
:105D20003F0B640DDB0F8D4218D08C4211D0002D3B
:105D300018D130438446002C1ED13A431CD163460F
:105D40000020002B30D05146022001390840013894
:105D50002AE039001143EAD0022025E03043FBD18C
:105D6000AC4226D0002C26D13A4324D15146022001
:105D700001390840013817E06246002A0FD09A45E1
:105D8000E1D1A54205DBBE42DDD819D00020BE42DC
:105D90000AD25046012301389843013004E0012221
:105DA000013B9343180001301CBC90469946A24623
:105DB000F0BD3A43D0D19A45C5D1A542C3DCE0E756
:105DC000C845C0D80020C845E3D3EDE7FF07000071
:105DD000F0B55746DE464E464546E0B583460600DA
:105DE0000F03480087B092461D003F0B400DCC0FBB
:105DF000002800D16FE0DE4B984238D08023FF00AE
:105E00001B041F43730F3B430193DA4B0027994652
:105E100000239B46F60081442B0369001B0B52466E
:105E20009846490DED0F002900D185E0D04B9942ED
:105E300000D173E04346DA0080231B04134352462B
:105E4000CC48520F84461343524600206144D2008E
:105E500089442100694000918C46012149448A46C9
:105E60000F2F00D990E0C449BF00CF59BF465B4611
:105E70003B43019300D06AE10223082700268146B4
:105E80009B46C9E732005846019B614600910228B3
:105E900000D175E0032800D1FEE1012800D02CE1FB
:105EA00000230027002600253F032A0D3F0BB3489F
:105EB00012053A4302401B051343009A5B00D107C9
:105EC0005B080B433000190007B03CBC9046994674
:105ED000A246AB46F0BD5B463B43019300D12FE1A8
:105EE000002F00D1A5E1380000F0EAFD03000B3BD4
:105EF0001C2B00DD96E11D22D31A5A460100DA4020
:105F00005E4608398F4013008E403B4301939C4B03
:105F100000271B1A994600239B467DE741465346BE
:105F20000B4393498C46E144002B00D01AE1022236
:105F30000220174300228CE7134300D10DE14346B2
:105F4000002B00D181E1404600F0BAFD02000B3A7F
:105F50001C2A00DD72E10100434608398B40984657
:105F60001D239A1A5346D3401A0043461343524600
:105F70008A404946081A824989468144002068E7D8
:105F80007B4B002700268EE7140C1204120C110024
:105F9000370C3604350C794328008C462E006043BC
:105FA0006044834656432100300C8046584679436E
:105FB00040440291844506D98846802149028C4696
:105FC000E044414602913604010C360C00048B4635
:105FD00081191E0C1B041B0C0391190079438C467C
:105FE000280075436544A8465843050C454477434B
:105FF000A94203D9802149028C466744290C8C466A
:1060000039000004000C2D042D186144AB440591A7
:106010005946049101990F043F0C080C3900514373
:106020004243904602008C46090C8B4662437C43F7
:1060300044445C44A04503D9802149028846424437
:10604000210C884661460904090C8C4639005943E5
:10605000434370437E430F0CF6182404BE19644476
:1060600042448C46B34203D980235B0298464044A5
:10607000029B61469846049B370443449B46AB45CC
:10608000AD416B420D0405992D0C8C467F19674478
:10609000FD18A8465D462D19A542A44193466442C9
:1060A000A446C344DC448F42BF4198459B4193457D
:1060B0009241A445A4415B427F421F43360C5242A9
:1060C0006442BF192243BF18624638184302D20DFA
:1060D000039913436A020A43501E82416146ED0D43
:1060E0002A434E023243D90100D4B3E001265008BE
:1060F00032400243DE0732435B08224C5444002CFA
:1061000062DD510709D00F201040042805D0101D72
:106110009042924152429B180200D90104D580243A
:106120001948E400034054441848844200DD27E73E
:106130005E075B02D2081F0B630516435B0DB2E6D8
:10614000002399460133042700269B4664E6032377
:10615000019781460C279B465EE6012201201743EA
:10616000002276E6032303201F43434671E6C04620
:10617000FF07000001FCFFFF8C910000FFFF0F8074
:106180000DFCFFFFFF030000FFFFFFFEFE07000006
:106190000023802700933F030026434B83E6019BA7
:1061A0003200A446584670E6AC466EE68027019958
:1061B0003F0339422DD03B422BD11F433F033F0BBE
:1061C00000951600384B6EE601252D1B382D00DD9D
:1061D00066E61F2D40DC35481C0050441600824006
:1061E0008440EE40501E824134431443EB4062072A
:1061F00009D00F222240042A05D02200141D944207
:10620000804140421B181A023ED501230027002678
:1062100049E68027019B3F031F433F033F0B009448
:10622000214B40E603005A46283B9A400026019243
:106230006DE6584600F044FC203057E60300524615
:10624000283B9A401300002293E6504600F038FCA9
:1062500020307BE6CA4650E71F201E004042041B48
:10626000E640202D03D0124C5444A3401A43501E44
:106270008241324307260027164009D00F20002311
:10628000104014000428B9D122005E075B021F0BE6
:10629000D2081643002306E680273F031F433F032F
:1062A0003F0B1600004BFEE5FF0700001E04000038
:1062B0003E040000F8B557464E464546DE460C0003
:1062C0000903E0B5490A460F5F0031431E03DB0FA7
:1062D000760A9B46530F3343C84E6500C000E40F57
:1062E000D2006D0DA24681467F0D9C469046B74276
:1062F00000D1B9E05B46012673409B46EE1BA345E7
:1063000000D183E0002E63DD002F00D0B1E06346B2
:10631000134300D123E1731E002B00D0BAE1861A8B
:106320006346B04280410125C91A4042091A0B0256
:1063300000D447E149024B0A98464346002B00D15E
:1063400089E1404600F0BCFB0300083B1F2B00DD49
:106350007CE120223000D21A4146D0409940020010
:106360009E400A439D4200DD6AE15D1B6B1C1F2BB2
:1063700000DD94E1202110003500C91A8E40DA407A
:106380008840DD40711E8E41110007222843002500
:1063900006433240002A09D00F233340042B05D096
:1063A000331DB342B641764289191E000B0200D458
:1063B0003DE26A1C914B55056D0D9A4200D119E1E1
:1063C0008F4AF6080A40570752023743120B9BE0E8
:1063D000002E00D0C5E06E1C7605760D012E00DC87
:1063E00048E16746861ACB1BB042BF417F42B846A0
:1063F0001F004346FF1A3B00B8461B0200D55FE171
:1064000037439AD100220024002579E0002E00DCD9
:10641000FAE0002F00D18DE0784B9D4267D08023B9
:1064200067461B041F43BC46382E00DC52E163461E
:1064300013435A1E93411E18864280414042091858
:106440000B0200D4BEE06D4B01359D4200D1D2E07D
:106450006B4A73080A4001210E401E435108D307BE
:1064600007221E43324095E71E00164300D045E741
:1064700040E7624B9D423AD0802367461B041F438E
:10648000BC46382E00DDEBE01F2E00DC3AE1330085
:106490006746203BDF403B00202E05D04027BF1B36
:1064A0006646BE40324390464646721E964133438E
:1064B000DAE0002B00D114E26346134300D168E117
:1064C00080234E07C008C9081B030643194208D0A1
:1064D0006046C008184204D163460100D2085E0736
:1064E0001643F3009946C900720F444D11434B46C1
:1064F000DE08424B4F073743CA089D4200D16EE089
:1065000012036D05120B6D0D00211203130B0A0D02
:1065100012051A433B4B2D0513402B435B00E40748
:106520005B082343380019003CBC90469946A246BC
:10653000AB46F8BD6346134311D0731E002B00D049
:1065400007E18618864280416144404209180125CE
:106550000B0237D502257BE73E00614691463500A8
:10656000C5E75C46002D00D0E1E00B000343F3D00B
:10657000731C00D1ACE1214B9F4200D13AE1F343BF
:10658000382B00DD6FE11F2B00DD8CE120250E0094
:10659000ED1AAE40B0460600AA46DE4045463543F9
:1065A0002E005546D940A8406346451EA8415B1AB7
:1065B0009C463043161AB242924163465242991A9F
:1065C0003D00B4E607223240002A00D0E4E60B4B3F
:1065D000F6084F073743CA089D4200D090E73B00BA
:1065E000134300D1A6E180231B031A431203120BAD
:1065F000024D89E715000022002785E7FF0700000C
:10660000FFFF7FFFFFFF0F80002E00D0C7E06B1C55
:106610005E05760D012E00DCF0E0C84DAB4200D1E6
:10662000B9E085180A0085428941624449425118FF
:106630000722CE076D082E43490832401D00A9E607
:10664000BF49ED1A114007223240A3E63200283834
:106650008240002686E6300000F032FA203073E6F1
:10666000634613435A1E9341C61AB04280414042CA
:10667000091A5CE60E00674606431743002D5ED1FB
:10668000002E00D0F3E0002F00D11EE15C466146F1
:1066900091462CE7A94FBE427BD01E00F1E61000C8
:1066A0001F3DE840202B03D04021CB1A9A401643CF
:1066B000731E9E410722064332400021002583E7D6
:1066C000161A6346B2428041591A40420B1A984644
:1066D0005C4632E61F2E00DDABE02027BB1B9A464E
:1066E00063465746BB40994613004F46F3401F434D
:1066F0003B005746BA40571EBA4113436246F24028
:10670000891898E62027BB1B9A4663465746BB402C
:10671000994613004F46F3401F433B005746BA408B
:10672000571EBA4113436246F240891A9CE7834BD5
:106730009F425FD080252D047342294320E7002E1D
:106740000CD1002F00D1D0E05C46614691467B4DD4
:10675000CDE67A4FBE421CD01E0065E6002F18D051
:10676000C0084E0706438020C9080003014208D034
:106770006346DC08044204D12100DA46D2085E07F1
:106780001643F300994601245346C900720F114382
:106790001C406A4DABE61D0000220027B4E6002D28
:1067A00059D10B00034300D1D6E6731C00D1B2E0EF
:1067B000624B9F421ED0F343382B6FDC1F2B00DD52
:1067C00097E020250E00ED1AAE40B0460600AA461E
:1067D000DE40454635432E005546A840D940451E6B
:1067E000A8418C440643B6189642924151426144F6
:1067F0003D0025E63D006146914678E60B000343E7
:10680000002D00D055E6002BF5D06346134300D190
:106810006DE6861886428041614440420918002294
:106820000B0200D4D0E6464B01351940B2E5B14623
:106830005DE633006746203BDF403B00202E05D05D
:106840004027BF1B6646BE40324390464646721EF6
:1068500096413343EFE5394B9F42CBD080252D0441
:1068600073422943A8E70843411E8841A2E6002F4E
:1068700000D13CE66346861ACF1AB0429B415B4288
:10688000FB1A98461B024ED5161A6346B242924135
:10689000591A5242891A5C4600227BE501430E00D8
:1068A000711E8E419FE71D000E00203DEE40B04658
:1068B000202B04D04025EB1A9940084381464846D6
:1068C0004346411E8841184374E60022002417E61F
:1068D000161A6346B2429241591A5242891A3D0031
:1068E00025E561469146154D01E6802200241203FC
:1068F00079E61D000E00203DEE40B046202B04D06E
:106900004025EB1A9940084381464E464346711E86
:106910008E411E4367E7861896429B4161445B4265
:10692000C9183D008CE547463743CED00722414683
:10693000324049E600273A00E6E5C046FF0700007E
:10694000FFFF7FFF70B50C4E0D031C0349005B0079
:106950002D0B490D240B5B0DB14208D006490020D8
:106960008B4203D114432000441EA04170BD054357
:106970000120002DFAD1F1E7FF07000030B5144DDA
:106980000A034B00120B5B0DC90F0024AB4211DD53
:10699000104CA34210DC8024640322430E4CE41A02
:1069A0001F2C0CDD0D48C31ADA4013005C4200298D
:1069B00000D11C00200030BD094BCC18FAE7094D6E
:1069C000E040AC4663449A4013000343EEE7C04600
:1069D000FE0300001D040000330400001304000047
:1069E000FFFFFF7FEDFBFFFF70B500282DD0C31721
:1069F000C5185D40C40F280000F062F8154B1B1A43
:106A00005B055B0D0A2815DD0B38854000222D0340
:106A10002D0B002110002D030A0D2D0B12052A430A
:106A20000D4D1B052A4013435B00E4075B0823431D
:106A3000190070BD02002900153291400A000B2197
:106A4000081AC5402D032D0BE3E700240023002581
:106A50000022DEE71E040000FFFF0F8010B5041EB9
:106A600025D000F02DF8144B1B1A5B055B0D0A288E
:106A700012DD0B38844000222403240B0021100077
:106A800024030A0D240B120522430C4C1B05224043
:106A900013435B00590810BD0200210015329140DC
:106AA0000A000B21081AC4402403240BE6E7002344
:106AB00000240022E2E7C0461E040000FFFF0F8012
:106AC0001C2101231B04984201D3000C10391B0A1E
:106AD000984201D3000A08391B09984201D30009E2
:106AE000043902A2105C40187047C0460403020239
:106AF00001010101000000000000000070B5002647
:106B00000C4D0D4C641BA410A64209D1002602F0C6
:106B1000C9F80A4D0A4C641BA410A64205D170BDE9
:106B2000B300EB5898470136EEE7B300EB589847AF
:106B30000136F2E7F4010020F4010020F401002006
:106B40000802002010B5034B0100186800F08EF811
:106B500010BDC0462400002010B5034B010018688A
:106B600000F03AF810BDC0462400002082B0002991
:106B700000D101A9101E06D0002B06D013780B609F
:106B80001078431E984102B0704702204042FAE755
:106B9000002310B59A4200D110BDCC5CC45401331F
:106BA000F8E710B5884202D98B18984203D3002326
:106BB00007E08B5C8354013AFBD210BDCC5CC4541B
:106BC00001339A42FAD1F8E703001218934200D138
:106BD000704719700133F9E770B50500002910D02E
:106BE0000C1F2368002B00DAE418280001F0C7FB13
:106BF0001D4A1368002B05D163601460280001F062
:106C0000BFFB70BDA34209D9216860188342F3D14C
:106C100018685B6841182160EEE713005A68002A83
:106C200001D0A242F9D919685818A0420BD12068A6
:106C30000918581819608242E0D11068526841184A
:106C400019605A60DAE7A04202D90C232B60D5E71D
:106C500021686018824203D110685268411821608F
:106C600062605C60CAE7C046400B0020032370B539
:106C7000CD1C9D43083506000C2D1ED20C25A942C3
:106C80001DD8300001F07BFB254A14682100002943
:106C900019D1244C2368002B03D1300000F0ACFC48
:106CA00020602900300000F0A7FC431C2BD10C23EE
:106CB0003000336001F064FB03E0002DDFDA0C23C9
:106CC0003360002070BD0B685B1B19D40B2B03D9FC
:106CD0000B60CC18256003E04B688C420DD113602B
:106CE000300001F04DFB200007220B30231D9043A4
:106CF000C31AE7D05A42E250E4E763600C00EFE7C2
:106D00000C004968C3E70323C41C9C43A042E1D0A4
:106D1000211A300000F070FC431CDBD1C7E7C046ED
:106D2000400B0020440B0020F0B58BB014001D1E5A
:106D3000129953DA802424061B191D0014002D23F8
:106D40000B702023149E03229E43462E07D033004F
:106D5000453B59424B411099013ACB18109309AB6E
:106D6000049308AB0393139B00920293109B2200A1
:106D700001932B0000F00CFD0700472E02D1119B60
:106D8000DB0724D5109BFB180793462E14D13B78C4
:106D9000302B0CD10022002320002900FEF7C4F87C
:106DA000002804D10123109A9B1A139A1360139B95
:106DB000079A1B68D318079300220023200029009C
:106DC000FEF7B2F8302200280DD0079B0993380057
:106DD000099B159ADB1B13600BB0F0BD0023AFE7D6
:106DE000591C09911A70099B07998B42F8D3EEE759
:106DF000F0B5831C85B0019306000C0002702B23B4
:106E0000002901DA2D234C427370092C22DD02ABDC
:106E1000DD1D20000A21FEF771F86F1E3031397038
:106E200020000A21FDF784FF040009280BDC023D45
:106E30003034019B2C7002AA07321800AA4204D8F1
:106E4000801B05B0F0BD3D00E3E72A7801351A70DC
:106E50000133F0E73023E418B370301DF470EFE72E
:106E6000F0B595B00C000A920B931A9D099001F0B1
:106E70006FFA036818000C9300F0F0FB00231293E4
:106E800023680E900D930D99277E2B680722C90564
:106E900045D59B1893431A0008322A601A685B682C
:106EA000A264E3640122E56CA66C6B005B080F939F
:106EB0005242AC4B30000F99FFF744FD002830D10F
:106EC0000122A84B524230000F99FEF73DF80028EE
:106ED00027D10022002330002900FEF72BF80028DC
:106EE00003D023002D2243331A709F4D472F00D823
:106EF0009E4D032300260D9A236101339A4322609D
:106F00000B9B13AA009321000A9B099800F0F4F947
:106F1000431C00D093E00120404215B0F0BD073380
:106F2000B8E732002B0030002900FFF70BFD0028E6
:106F300004D08F4D472FDCD88E4DDAE780230D9992
:106F40006268DB000B43511C43D10732626012AA16
:106F50000021059211AA0392232223600691019336
:106F600008A9636852180292009332002B0004971C
:106F70000998FFF7D9FE20233A0005009A43472AD3
:106F800007D1119BDA1C02DB6268934245DD023FA8
:106F9000FFB21199652F25D8200001393A005030F1
:106FA0001191FFF725FF129A060013182361012A99
:106FB00002DC2268D20701D501332361232308AA0A
:106FC0009B181B78002B9BD023002D2243331A7073
:106FD00096E7672F00D176E1472FB8D1002AB6D1C6
:106FE0000122B3E7662F19D1636800290CDD216106
:106FF000002B02D12268D20702D501335B1823612E
:10700000119B0026A365D9E7002B03D1012221683B
:10701000114200D09A1C2261F2E76727119B129A55
:10702000934205DB22682361D207E9D50133E6E705
:107030000121002B01DC4918C91A5218EBE722681C
:10704000530508D423692A000A9909980B9DA8477B
:10705000431C29D15FE7652F00D8E0E0A06CE16C0C
:1070600000220023FDF760FF002834D00123424AAC
:107070000A9909980B9DA847431C00D14BE7119B27
:10708000129A934202DB2368DB070DD50B9D0E9B02
:107090000C9A0A990998A8470025431C00D13AE7A1
:1070A000129B013BAB420ADC23689B0700D508E139
:1070B000139BE068984200DB2FE718002DE72200C1
:1070C00001231A320A9909980B9EB047431C00D13C
:1070D00021E70135E4E7119B002B2DDC0123264A33
:1070E0000A9909980B9EB047431C00D113E7119BE6
:1070F000002B05D1129B002B02D12368DB07D3D5CF
:107100000B9E0E9B0C9A0A990998B0470026431CC7
:1071100000D100E7119B5B42B34201DC129B92E776
:10712000220001231A320A9909980B9FB847431C81
:1071300000D1F0E60136EDE7A36D129F9F4200DD1E
:107140001F00002F08DD3B002A000A9909980B9EBA
:10715000B047431C00D1DEE600230D93FB43DB1751
:107160000F9318E0FFFFEF7FDA910000D691000047
:10717000E2910000DE910000E69100002200012370
:107180001A320A9909980B9EB047431C00D1C2E6F7
:107190000D9B01330D930F9BA66D0D9A3B40F31A87
:1071A0009342EBDC119B129AAD19934210DB2368DA
:1071B000DB070DD4129F119BBE1BFF1AB74200DDE7
:1071C0003700002F0DDCFE43F31700250C931CE065
:1071D0000E9B0C9A0A9909980B9FB847431CE9D15A
:1071E00099E63B002A000A9909980B9DA847431C81
:1071F000E9D190E6220001231A320A9909980B9EE0
:10720000B047431C00D186E60135119A129B0C99B8
:107210009B1A3A000A409B1AAB42EBDC44E7129BF4
:10722000012B02DC01231A4232D001232A000A99E1
:1072300009980B9FB847431C00D16CE60E9B0C9A33
:107240000A9909980B9F0135B847431C00D162E6A3
:10725000A06CE16C129B00225F1E0023FDF764FE10
:107260003B00002814D000250AE0220001231A3236
:107270000A9909980B9FB847431C00D14BE601358A
:10728000129B013BAB42F0DC220033005032DBE6C4
:107290002A000A9909980B9DA847431CF4D13AE6A5
:1072A0002200012319320A9909980B9EB047431C0A
:1072B00000D130E60135E368139A9B1AAB42EFDC4C
:1072C000F6E60025F7E7002A00D189E600210691BD
:1072D00012A9059111A90391232108A80918236077
:1072E000019300922B000497029132000998FFF756
:1072F0001BFD050045E6C046F7B5150001938A68F9
:107300000B6900900C00934200DA130022002B60FE
:1073100043321278002A01D001332B6023689B0688
:1073200002D52B6802332B60062723681F4027D025
:10733000230043331B785A1E93412268920630D4AF
:107340002200019943320098089EB047431C25D083
:10735000062320682A68E16803400025042B03D136
:107360008D1AEB43DB171D40A3682269934201DDB0
:107370009B1AED180027BD4220D1002010E00137F4
:10738000E3682A689B1ABB42D2DD2200012319322E
:1073900001990098089EB047431CF0D1012040425B
:1073A000FEBD3020E1184331087021005A1C4531E0
:1073B0000978A218433202331170C1E72200012379
:1073C0001A3201990098089EB047431CE6D0013755
:1073D000D1E70000F0B589B004920A00433205936A
:1073E000039002920A7E0C000E9B6E2A00D186E06A
:1073F0001FD8632A33D008D8002A00D18CE0582A3D
:107400004DD0250042352A7030E0642A01D0692A27
:10741000F7D1196825680A1D280629D508681A6059
:10742000002803DA2D23029A404213706B4E0A277C
:107430004FE0732A74D008D86F2A1FD0702AE0D189
:10744000202209680A43226003E0752A16D0782AB0
:10745000D7D12200782145321170614E22E02500FB
:107460001A684235111D196013682B70012365E0FD
:1074700008681A606906D3D500B2D1E71968256893
:10748000081D186008682E0605D5544E08276F2A77
:107490001BD00A2719E06D06F7D580B2F5E7453114
:1074A0004E4E0A7018682268011D006819601506A2
:1074B00021D5D30702D520231A43226010270028A4
:1074C00003D1202322689A43226023000022433301
:1074D0001A706368A360002B58DB04222168914373
:1074E0002160002854D1029D002B5AD0250033780A
:1074F00042352B7055E05506DBD580B2D9E71A68C6
:107500000D68101D4969186013682E0601D51960B1
:1075100002E06D06FBD519800023029D23614FE038
:107520001A68111D1960156800216268280000F0B2
:107530001BFF002801D0401B6060636823610023AB
:10754000029A13703CE023692A0004990398059D70
:10755000A847431C3ED023689B0715D4079BE068CF
:10756000984239DA180037E02200012319320499D1
:107570000398059EB047431C2CD00135E368079A59
:107580009B1AAB42F0DCE9E70025F7E70028ADD015
:10759000029D3900FDF7C8FB735C013D2B7000288C
:1075A000F7D1082F09D12368DB0706D56368226964
:1075B000934202DC3023013D2B70029B5B1B236155
:1075C000059B07AA00932100049B0398FFF794FEF4
:1075D000431CB8D10120404209B0F0BDE891000041
:1075E000F991000010B5034B0A000100186801F082
:1075F000BDF910BD24000020002370B5064C050025
:107600000800236001F040FB431C03D12368002BDA
:1076100000D02B6070BDC0464C0B00200EB400B5EE
:107620000B499CB01DAB029006900791049109484C
:10763000094904CB0591006802A9019301F01EFAE3
:107640000023029A13701CB008BC03B01847C04650
:10765000FFFFFF7F240000200802FFFF0023C25C21
:107660000133002AFBD1581E70470B1E04D0FF2A9D
:1076700004D98A2303608B3B180070470A700123EA
:10768000FAE7F0B503690C6989B007000591002697
:10769000A34265DB0B00013C1433A50003935B1987
:1076A00004930300143302935D19049B28681B683C
:1076B000591C0193FDF7B2FA0190B04229D0039B07
:1076C00002989C460696624608CA9446019A99B268
:1076D00051431B0C534389190A0C9B1807931E0C2A
:1076E000036889B29AB2069BD2180368521A190C21
:1076F0006B469B8BCB1A11145B18191492B21B04A6
:107700001A43049B069104C06345DCD22B68002B0E
:107710002DD00599380001F049F800281FDB00251D
:10772000019B0298013303990193026808C992B240
:1077300055199AB2AA1A05681B0C2D0CEB1A1514D0
:107740005B191D1492B21B04134308C0049B8B42A7
:10775000EBD2029AA300D3181A68002A11D0019E16
:10776000300009B0F0BD2B68002B04D1013C029B16
:10777000043DAB42F7D33C61CBE71A68002A04D141
:10778000013C029A043B9A42F7D33C61E7E70000D0
:10779000F0B516001F00446A9BB00290239D069628
:1077A0000797002C08D11020FFF7CCF9029B5862F4
:1077B000446084600460C460029B5B6A19680029AD
:1077C0000BD05A68012393404A608B60029800F006
:1077D00010FE0022029B5B6A1A60002F20DA012350
:1077E0002B607B005B080793079CB24B220017932A
:1077F0001A409A4217D1B04B229A1360069B002B75
:1078000003D1240301D100F087FDAC4B249A0893E7
:10781000002A02D0AA4B249A136008981BB0F0BD2E
:1078200000232B60E0E7069E079F00220023300024
:107830003900FDF779FB051E0BD00123229A136056
:10784000A04B249A0893002AE7D09F4A24990A6003
:10785000E3E718AB019319AB009332003B000298A9
:1078600001F022F8630003905B0D74D03A03974C4B
:10787000120B14432100964A300016959E180022E0
:10788000944BFEF717FD944A944BFEF7A1FA944AE5
:10789000944BFDF777FB040030000D00FFF7A4F8D0
:1078A000914A924BFEF794FA02000B002000290047
:1078B000FDF768FB04000D00FFF760F800220700E9
:1078C000002320002900FDF735FB002809D03800EF
:1078D000FFF78AF82B002200FDF726FB43425841B0
:1078E0003F1A01231493162F0DD88149FB00C918A4
:1078F00008684968069A079BFDF730FB002846D0C8
:107900000023013F1493189B9E1B00230A9333000E
:10791000013B0B9304D501239B1B0A9300230B937C
:10792000002F36DB0B9B1197DB190B93002304937D
:10793000209B0124092B00D984E0052B02DD0024C3
:10794000043B2093209B981E032800D984E0FDF778
:107950005BF97577286A189B199A9E18654BF2187F
:10796000202A0FDD40239B1A9C40634B0698F31896
:10797000D8402043FFF772F80123604C013E0919FB
:1079800016937CE7202306989B1A9840F2E7149000
:10799000B9E70A9BDB1B0A937B42049300231193F4
:1079A000C6E701230D93219B002B59DD0C9309930E
:1079B000029A556A00226A60043210001430696825
:1079C000984252D9029800F0DCFC029B28605B6A66
:1079D0001B680893099B0E2B00D90AE1002C00D1EB
:1079E00007E1069B079C12931394002F00DC89E0AB
:1079F0000F213A003E4B0A40D2009B181D685E687A
:107A000002233C110E93E3060BD53D4B0C401A6A42
:107A10005B6A12981399FDF7D1FD03230690079135
:107A20000E9300233AE001230D93219BFB180C9346
:107A300001330993002BBBDC0123B9E70023B1E735
:107A40000023F1E700230D942093013B00220C93C7
:107A5000099313332192ABE701230D93023BF5E722
:107A600001230C9309931A00F4E701316960520075
:107A7000A3E701231C420ED00E9B214A01330E9333
:107A8000109B2800DB009B1831001A685B68FEF72A
:107A90009FF905000E00109B641001331093002C19
:107AA000E7D1069807992A003300FDF787FD069075
:107AB000079142E00000F07F0F27000014930000C0
:107AC00017930000E6910000E79100000000F03FEE
:107AD00001FCFFFF0000F83F61436F63A787D23FBF
:107AE000B3C8608B288AC63FFB799F501344D33FAD
:107AF000409300003204000012040000000010FE59
:107B00001893000002230E93002F16D01298139999
:107B10007C420D332340CE4ADB00D3181A685B68E1
:107B2000FEF756F9002301261D0006900791241147
:107B3000002C00D08CE0002BB9D1149B002B00D17D
:107B400096E0069C079D0022C24B20002900FDF70D
:107B5000F1F9002800D18BE0099B002B00D187E0D0
:107B60000C9B002B41DDBC4B002220002900FEF7BE
:107B70002FF90E9B0690079101330E930C9B7E1EEE
:107B80000E981093FEF730FF069A079BFEF720F938
:107B90000022B24BFDF7F6F9B14A0E900F910E9C00
:107BA0000F9D94460F9B634415931D00109B002B63
:107BB00061D1069807990022AA4BFEF77BFB2200B1
:107BC000159B06900791FDF7C9F9002800D0A8E29F
:107BD000A5480F99844661440B0006980799220036
:107BE000FDF7A8F9002800D095E2129B139C06939C
:107BF0000794199B002B00DA5CE10E2F00DD59E1A0
:107C0000934BFA009B185C681B6804930594219BB6
:107C1000002B00DBD8E0099B002B00DDD4E000D076
:107C20007DE20498059900228E4BFEF7D1F8069A62
:107C3000079BFDF79DF9099B04931E00002800D0C7
:107C40004FE2089B089A5D1C3123013713704BE209
:107C500034420AD00E9B854A01330E93EB009B18E9
:107C60001A685B68FEF7B4F83300641001355FE70B
:107C70003E00099B84E7109B0D995A1E744BD2005D
:107C80009B181A685B68002949D000207849FDF7E5
:107C900095FC2B002200FEF70DFB089B0E900F9128
:107CA000159306980799FEF769FE0400FEF79CFEFF
:107CB00002000B0006980799FEF7FCFA159B30347A
:107CC0005D1C1C700E9A0F9B06900791FDF732F910
:107CD00000286CD1069A079B00205E49FEF7EAFA5D
:107CE0000E9A0F9BFDF726F9002800D0C3E0089BF1
:107CF000109AEB1A9A4200DC77E70E980F9900224F
:107D0000554BFEF765F800220E900F9106980799E3
:107D1000514BFEF75DF8159506900791C1E72000DD
:107D20002900FEF755F8089C109A230094460E90FF
:107D30000F916344159306980799FEF71FFE0500FF
:107D4000FEF752FE0B00020006980799FEF7B2FA02
:107D50003035159B2570013406900791A3422AD136
:107D60000E980F99089A109B9446634400221D00B8
:107D70003F4BFDF707F902000B0006980799FDF746
:107D8000EDF8002800D076E00E9A0F9B00203849CD
:107D9000FEF790FA02000B0006980799FDF7CAF863
:107DA000002800D121E76B1E1A78302A01D0370055
:107DB0003FE01D00F7E7069807990022264BFEF7E3
:107DC00007F806900791B6E7089E049A059B069867
:107DD0000799FDF7F3FBFEF7D1FD0400FEF704FE63
:107DE000049A059BFDF7F4FF02000B000698079923
:107DF000FEF760FA230030333370099A089B751C34
:107E0000EB1A9A4248D102000B00FDF7BBF8049A26
:107E1000059B06900791FDF7A1F800282AD1049A46
:107E2000059B06980799FDF77FF8002801D0E30726
:107E300020D40399029800F0DCFA00232B70229BD7
:107E400001371F60249B002B00D1E6E41D60E4E4B1
:107E5000409300000000F03F0000244000001C4060
:107E60000000C0FC000014400000C07C189300001B
:107E70000000E03F3E006B1E1A78392A06D1089AAE
:107E80009A4207D130231370130001361A78013259
:107E90001A708CE71D00EEE70022A44BFDF798FF57
:107EA00000220023069007912E00FDF73DF80028E0
:107EB0008BD0BEE70D9A002A00D1DAE0209A012A81
:107EC00000DDBDE0169A002A00D1B5E0984A9B1863
:107ED000049D0A9C0A9A0121D2180A920B9A0298D0
:107EE000D3180B9300F025FB0600002C0EDD0B9B36
:107EF000002B0BDD0B9A2300944200DD13000A9A3D
:107F0000E41AD21A0A920B9AD31A0B93049B002BF1
:107F10001FD00D9B002B00D1AFE0002D11D0310000
:107F20002A00029800F09EFB039A010006000298C6
:107F300000F008FB03991090029800F05AFA109B89
:107F40000393049B5A1B04D00399029800F08AFB08
:107F500003900121029800F0ECFA119B0490002B91
:107F600000D1E3E11A000100029800F07BFB209BA6
:107F70000490012B00DD82E00025069BAB420ED170
:107F8000079B1B03AB420AD1179B079A134206D0EB
:107F90000A9B013501330A930B9B01330B93119B11
:107FA0000120002B6CD10B9B18181F2318407ED08A
:107FB00001331B1A042B70DD1C23181A0A9B24188A
:107FC0001B180A930B9B1B180B930A9B002B05DDB8
:107FD0001A000399029800F097FB03900B9B002B6B
:107FE00005DD1A000499029800F08EFB0490149BA2
:107FF000002B5ED00499039800F0D8FB002858DAD3
:1080000000230A220399029800F00CFA0D9B013F0D
:108010000390002B00D190E1002331000A22029846
:1080200000F000FA0C9B0600002B00DD88E0209B8E
:10803000022B00DC84E044E03623189A9B1A47E7C1
:10804000099B5D1E049BAB4208DB5D1B099B002B5B
:108050000CDA0A9B099A9C1A00233BE7049B0495BF
:10806000EA1A119B00259B181193EFE70A9C099BC4
:1080700030E7049D0A9C0D9E37E7049A64E70025CB
:10808000049B049A1B69109303339B00D318586810
:1080900000F006FA2023181A85E7042B95D00A9AD7
:1080A0001C33D2180A920B9AE418D3188CE70300F9
:1080B000F5E7099B002B3DDC209B022B3ADD099B59
:1080C0000C930C9B002B0CD104990522029800F014
:1080D000A9F904900100039800F068FB002800DD76
:1080E000AFE5219B089DDF43002309930499029883
:1080F00000F07FF9002E00D19BE6099B002B05D0F4
:10810000B34203D01900029800F073F931000298CD
:1081100000F06FF98DE6109B04931E00E1E7002349
:10812000FAE7109B370004931E008AE50000244004
:10813000330400000D9B002B00D1B2E0099B0C938F
:10814000002C05DD31002200029800F0DDFA060067
:108150003000002D11D07168029800F012F9310042
:10816000040033690C319A1C92000C30FEF710FDAC
:1081700001222100029800F0C7FA09960600089B28
:108180000A9304990398FFF77CFA09990D9004006B
:10819000039800F00BFB320010900499029800F055
:1081A0001FFB01230B93C36830340500002B04D15F
:1081B0000100039800F0FAFA0B902900029800F0F1
:1081C00018F90B9B209A13430ED1069A01331342E0
:1081D0000AD1392C26D0109B002B01DD0D9C3134A7
:1081E0000A9B5D1C1C7081E7109B002B07DB1D00A8
:1081F000209B1D4322D10123069A13421ED10B9BC3
:10820000002BEDDD03990122029800F07DFA04991C
:10821000039000F0CBFA002802DCE1D1E307DFD5C0
:10822000392CDBD10A9B0A9A5D1C392313706B1E13
:108230001A78392A67D001321A7057E70A9B5D1CF9
:108240000B9B002B04DD392CECD001340A9BC9E7D1
:108250000A9B0C9A1C70089BEB1A93423ED0002399
:108260000A220399029800F0DDF8099B0390B342BB
:1082700009D100230A220999029800F0D3F8099045
:1082800006000A957DE7099900230A22029800F06A
:10829000C9F8002309900A223100029800F0C2F8C0
:1082A000EEE7099B0C93089B069304990398FFF74C
:1082B000E8F9069B30305D1C18700C9A089B04008E
:1082C000EB1A9A4208DD00230A220399029800F073
:1082D000A9F806950390E8E7002309930399012282
:1082E000029800F011FA0499039000F05FFA002858
:1082F0009DDC01D1E3079AD46B1E1A78302A00D096
:10830000F4E61D00F8E7089A9A4203D131230137B9
:108310001370EBE61D008AE70B4B249A08930B4B76
:10832000002A01D0FFF777FAFFF777FA209B012B9D
:1083300000DC21E6119D012035E60C9B002BB2DC10
:10834000209B022BAFDDBCE60B93000013930000D3
:10835000034B1B68186A002800D10248F0307047B0
:108360002400002088000020C9B28218904201D168
:108370000020704703788B42FBD00130F6E770474E
:10838000704770B5466A04000D00002E07D110201A
:10839000FEF7D8FB6062466086600660C660666A6B
:1083A000F368002B13D0636AAA00DB689B18186877
:1083B000002818D101210E00AE40721D920020004D
:1083C00000F0C6FA00280CD0456086600DE021223E
:1083D0000421200000F0BCFA636AF060DB68002B27
:1083E000E1D1002070BD02681A6000230361C36000
:1083F000F8E770B5446A06000D00002C07D1102084
:10840000FEF7A0FB7062446084600460C460002DCD
:1084100007D0736A6A68DB6892009B181A682A6042
:108420001D6070BDF7B51E0014239C4607000C00AC
:1084300000200D698C4463461B68013099B2634685
:108440001B6851431B0C534389190E0C9B1989B2AD
:108450001E0C1B045B18614608C18C468542EADC91
:10846000002E1BD0A368AB4212DC63683800591C95
:10847000FFF787FF2100236901909A1C92000C31BD
:108480000C30FEF785FB21003800FFF7B2FF019C9E
:108490002B1D9B00E31801355E6025612000FEBDA9
:1084A0000300020C0020824201D11B0410301A0E7E
:1084B00001D108301B021A0F01D104301B019A0FA1
:1084C00001D102309B00002B03DB01305B0000D4A4
:1084D000202070470722036810B501001A400DD014
:1084E00001240020234205D10230034203D0E3409F
:1084F00020000B6010BD9B080B60FBE79CB21000D6
:10850000002C01D110201B0CDAB2002A01D1083056
:108510001B0A1A0701D104301B099A0701D1023046
:108520009B08DA07E8D45B0801D00130E4E720209B
:10853000E0E710B50C000121FFF723FF01234461A0
:10854000036110BDF0B50B691400126989B00D000C
:10855000934201DA25000C002F6926696968BB196E
:108560000293AB68BA19934200DA0131FFF709FFB1
:108570000200BB1914329B00D3189C460021130043
:10858000049063451DD31435BF00EB191434B600B5
:108590000593A319039501940793079B01999942A9
:1085A00011D3029B002B06DD04235B429C446346EF
:1085B0001B68002B51D0049B029A18001A6109B065
:1085C000F0BD02C3DDE7019B1B6898B200281CD0F8
:1085D00015000026039F02CF2C688BB24343090C81
:1085E0004143A4B21B199B190E0029680695090C7A
:1085F00071181E0C89190E0C9BB209040B4308C597
:10860000059BBB42E7D8069B5E60019B1B681D0C67
:108610001ED0100000271368039E3168046889B2D9
:108620006943240C0919C9190F049BB23B43036029
:1086300080CE43683F0C6F439BB2FB18090C5B185C
:10864000059906901F0C0430B142E6D806994B609C
:10865000019B0432043301939FE7029B013B029389
:108660009FE700000323F7B5134005000E00140038
:10867000002B08D02249013B9A00525800233100B8
:10868000FFF7D0FE0600A310019336D06C6A002CD1
:1086900007D11020FEF756FA6862446084600460D7
:1086A000C4606F6ABC68002C07D116492800FFF728
:1086B00040FF00230400B86003600122019B1342C5
:1086C0000AD0310022002800FFF73CFF07003100EC
:1086D0002800FFF78EFE3E00019B5B1001930CD03B
:1086E0002068002807D1220021002800FFF72AFF78
:1086F0000023206003600400DFE73000FEBDC046B9
:108700000894000071020000F0B50D0017002B69FD
:10871000541185B0E3180193013300934968AB68A5
:108720000290009A934235DB0298FFF72AFE00235D
:108730000200060019001432A3422EDBE343DB17CC
:108740001C402B00A40014192A69143392009A18B3
:1087500094461F22174024D00132D21B03920022DC
:1087600019682000B9400A4304C404CB0399CA40E5
:108770009C45F5D84260002A02D0019B0233009349
:10878000009B0298013B33612900FFF732FE300065
:1087900005B0F0BD01315B00C3E798001150013313
:1087A000CAE704CB04C49C45FBD8E9E70A6903691E
:1087B00030B59B1A0DD192001430143184188918E9
:1087C000043C043925680A68954204D00123954287
:1087D00004D3180030BDA042F2D3FAE75B42F8E7B9
:1087E000F0B50D0085B00700110028001400FFF758
:1087F000DDFF061E08D101003800FFF7C2FD01238E
:108800004661036105B0F0BD01230193002804DB3C
:1088100023002C001D000023019361683800FFF73E
:10882000B0FD2F000022019B2669C3601434B30001
:10883000E31802932B6914379B00FB180393030082
:108840009446143320CC04CF0192AAB294446A46D1
:10885000614692882D0C8A1A0199090C691A15141F
:1088600049190D1492B209040A431A60039AAC46DE
:108870000433BA42E6D802991A008C4205D3043A6E
:108880001368002B0ED00661BCE704CC91B26144A2
:108890000D14120C5219151489B212040A43AC4675
:1088A00004C3E8E7013EEAE7F7B51D000121140023
:1088B000089FFFF766FD2B036D0006001B0B6D0D77
:1088C00024D10193002C27D068460094FFF702FEC4
:1088D000009C00281ED0019B20211A00091A8A4002
:1088E000C340224372610193019CB461631E9C41A9
:1088F00001343461002D18D0124BED1835232D189A
:108900003D60181A099B18603000FEBD802252039A
:108910001343D6E77461E7E701A8FFF7DBFD012405
:10892000019B346173612030E4E7074BC018074BAB
:108930003860E3189B00F3185869FFF7B1FD640134
:10894000201ADFE7CDFBFFFFCEFBFFFFFFFFFF3F5E
:108950004A4370B511001400FEF788F9051E03D0D4
:1089600022000021FEF730F9280070BDF8B507009D
:108970000D001600002905D11100FEF777F904005B
:108980002000F8BD002A03D1FEF726F93400F7E7EE
:1089900000F072F92C00B042F2D231003800FEF73C
:1089A00065F9041EECD029003200FEF7F1F8290029
:1089B0003800FEF711F9E3E7F0B58E6885B00700DF
:1089C0000C00039201939E423CD890238A89DB00DD
:1089D0001A4234D00325096923685B1A029363693C
:1089E00002985D43EB0F5D19019B6D1001331B185D
:1089F000AB4200D91D00530532D529003800FEF7DF
:108A000035F9061E09D10C233B6040230120A289C1
:108A100040421343A38105B0F0BD029A2169FEF7DD
:108A2000B7F8A389144A1A4080231343A381029BF9
:108A30002661F61826606561019EED1AA560019B0E
:108A40009E4200D9019E320003992068FEF7A9F8E2
:108A5000A36800209B1BA36023689E192660DAE7A9
:108A60002A003800FFF782FF061EE0D12169380096
:108A7000FEF7B2F8C7E7C0467FFBFFFFF0B59FB037
:108A8000029005938B890F0016001B0611D50B6908
:108A9000002B0ED14021FEF7E9F83860386100283C
:108AA00005D10C23029A013813601FB0F0BD40239A
:108AB0007B61002306AC6361203363761033A376B9
:108AC00035002B78002B01D0252B46D1AB1B04930E
:108AD0000CD0320039000298FFF76EFF431C00D122
:108AE000AEE06269049B9446634463612B78002B7B
:108AF00000D1A5E0012200235242626002A9543253
:108B000052186E1C2360E360A3601370A365317874
:108B100005225448FFF728FC751C00281FD1226845
:108B2000D30604D5532302A95B182021197013071B
:108B300004D5532302A95B182B21197033782A2BF3
:108B400016D0350000210A20E3682A786E1C303ADE
:108B5000092A4ED9002918D010E00135B1E7414B60
:108B60002268C01A01238340134323602E00CEE7FE
:108B7000059B191D1B680591002B01DB099304E07F
:108B80005B42E3600223134323602B782E2B0AD130
:108B90006B782A2B35D1059B02351A1D1B6805926F
:108BA000002B2BDB0793304E297803223000FFF790
:108BB000DBFB002806D04023801B83402268013560
:108BC000134323602978062228486E1C2176FFF77C
:108BD000CBFB00283CD0264B002B25D10722059B40
:108BE00007339343083305936369039A9B186361C2
:108BF00066E7434301219B183500A6E701235B424A
:108C0000D0E700230A201A000135636029786E1C22
:108C10003039092903D9002BC5D00792C3E7424355
:108C2000012352183500F1E705AB00933A00114BD0
:108C300021000298FEF714F90390039B0133D3D16E
:108C4000BB890B985B0600D42FE7012040422CE73C
:108C500005AB00933A00074B21000298FEF7BAFBE0
:108C6000EAE7C046149400001A9400001E94000025
:108C7000616E0000B98900000B1F1B68181F002BD4
:108C800001DA0B58C0187047044A1368002B00D152
:108C9000034B1818106018007047C046480B00209E
:108CA000500B0020F8B5C046F8BC08BC9E46704783
:108CB000F8B5C046F8BC08BC9E467047436C6F735D
:108CC0006520426C696E6420456E6420506F736944
:108CD00074696F6E3A20004F70656E20426C696E49
:108CE0006420456E6420506F736974696F6E3A201A
:108CF0000025000000000000160000000800000031
:108D00001C000000FF00000400040600000000003A
:108D100017000000080000001C000000FF00010414
:108D200001040700000000000A0000000800000025
:108D30001C000000120000010001FF000000000004
:108D40000B000000080000001C00000013000101DF
:108D50000101FF00010000000A00000008000000FF
:108D60001C000000FF00000500050A0001000000D3
:108D70000B000000080000001C000000FF000105BF
:108D800001050B00000000001400000008000000B6
:108D90002C000000FF0002000200040000000000A0
:108DA00015000000080000002C000000FF00030078
:108DB0000300050000000000100000000200000099
:108DC0001C000000FF000002000200000000000084
:108DD000110000000200000004000000FF00FFFF7F
:108DE000FFFF01000000000013000000020000006F
:108DF0001C000000FF0001030103FF000000000051
:108E000008000000030000001C000000100000002B
:108E10000000100000000000090000000300000036
:108E2000040000001100FFFFFFFFFF000100000031
:108E3000170000000300000004000000FF00FFFF17
:108E4000FFFFFF000100000016000000030000000B
:108E500004000000FF00FFFFFFFFFF000000000014
:108E60000200000001000000060000000000FFFFFB
:108E7000FFFFFF00010000000200000001000000F1
:108E8000040000000A00FFFFFFFF020001000000D5
:108E90000300000001000000040000000B00FFFFC1
:108EA000FFFF0300000000000400000001000000BC
:108EB0001C000000040000000000FF000000000093
:108EC00005000000010000001C000000050001007A
:108ED0000100FF000000000006000000010000008B
:108EE000040000000600FFFFFFFFFF00000000007D
:108EF0000700000001000000040000000700FFFF61
:108F0000FFFFFF0000000000180000000600000046
:108F100000000000FF00FFFFFFFFFF000000000057
:108F2000190000000600000000000000FF00FFFF25
:108F3000FFFFFF000000000012000000080000001A
:108F400004000000FF00FFFFFFFFFF000000000023
:108F5000030000000800000004000000FF00FFFF05
:108F6000FFFFFF00000000000C00000003000000F5
:108F700000000000FF00FFFFFFFFFF0000000000F7
:108F80000D0000000300000000000000FF00FFFFD4
:108F9000FFFFFF00000000000E00000008000000BE
:108FA00000000000FF00FFFFFFFFFF0000000000C7
:108FB0000F0000000300000000000000FF00FFFFA2
:108FC000FFFFFF00000000001B0000000800000081
:108FD00000000000FF00FFFFFFFFFF000000000097
:108FE0001C0000000800000000000000FF00FFFF60
:108FF000FFFFFF0001000000080000000800000063
:1090000000000000FF00FFFFFFFFFF000100000065
:10901000090000000800000000000000FF00FFFF42
:10902000FFFF090000000000000000000800000031
:1090300000000000FF00FFFFFFFFFF000000000036
:10904000010000000800000000000000FF00FFFF1A
:10905000FFFFFF0000000000000000006130000082
:10906000993200005D3000007D3200005D3200006A
:10907000D5320000B9320000593000005B300000EA
:1090800049320000F93200008B32000075300000D8
:10909000DD2F0000A131000005300000F0FFFFFFD0
:1090A000000000003932000091310000213300003F
:1090B00049300000000000000000000055350000AD
:1090C0005B410000334100003F410000BD33000020
:1090D000BF330000AD34000041726475696E6F20CB
:1090E0004D4B523130303000040309044172647535
:1090F000696E6F204C4C430012010002EF020140E8
:1091000041234E8000010102030100000000000025
:1091100000000000B9460000A548000043430000DD
:109120008F4300003D4300005547000053430000BB
:109130002D430000ED4300006B4300002943000075
:109140000D0A00252525642E256466006058000060
:10915000D2560000165700007A560000165700003D
:1091600006580000165700007A560000D25600003C
:10917000D2560000065800007A56000072560000D1
:10918000725600007256000014580000885F0000FC
:109190008A5E00008A5E0000A8610000845E000014
:1091A000845E000090610000A8610000845E000001
:1091B00090610000845E0000A86100009E610000D4
:1091C0009E6100009E610000AC6100004300504FB2
:1091D000534958002E00494E4600696E66004E41C4
:1091E0004E006E616E003000303132333435363728
:1091F0003839414243444546003031323334353604
:1092000037383961626364656600002020202020C1
:109210002020202028282828282020202020202026
:109220002020202020202020202020881010101016
:10923000101010101010101010101004040404046A
:109240000404040404101010101010104141414196
:10925000414101010101010101010101010101017E
:109260000101010101011010101010104242424290
:10927000424202020202020202020202020202024E
:109280000202020202021010101020000000000072
:1092900000000000000000000000000000000000CE
:1092A00000000000000000000000000000000000BE
:1092B00000000000000000000000000000000000AE
:1092C000000000000000000000000000000000009E
:1092D000000000000000000000000000000000008E
:1092E000000000000000000000000000000000007E
:1092F000000000000000000000000000000000006E
:109300000000000000000000000000496E66696E69
:10931000697479004E614E000080E03779C34143A3
:10932000176E05B5B5B89346F5F93FE9034F384DCB
:10933000321D30F94877825A3CBF737FDD4F157577
:10934000000000000000F03F00000000000024408A
:1093500000000000000059400000000000408F4065
:10936000000000000088C34000000000006AF840D0
:109370000000000080842E4100000000D0126341F4
:109380000000000084D797410000000065CDCD416A
:10939000000000205FA00242000000E8764837424B
:1093A000000000A2941A6D42000040E59C30A242E9
:1093B0000000901EC4BCD64200003426F56B0C435E
:1093C0000080E03779C3414300A0D8855734764305
:1093D00000C84E676DC1AB43003D9160E458E14366
:1093E000408CB5781DAF154450EFE2D6E41A4B44DB
:1093F00092D54D06CFF08044F64AE1C7022DB54420
:10940000B49DD9794378EA440500000019000000B2
:109410007D000000232D302B2000686C4C00656619
:0C94200067454647000000000000000007
:10942C000F00000040420F000A0000000A0000007C
:10943C00FFFFFFFFFFFFFFFF00C20100000008005D
:10944C00FFFFFFFF280000200000000000000000CC
:10945C000000000000000000000000000000000000
:10946C0000000000000000000000000000000000F0
:10947C0000000000000000000000000000000000E0
:10948C0000000000000000000000000000000000D0
:10949C0000000000000000000000000000000000C0
:1094AC00000000000000000043000000000000006D
:1094BC0000000000000000000000000000000000A0
:1094CC00000000000000000043000000000000004D
:1094DC000000000000000000000000000000000080
:1094EC00000000000000000043000000000000002D
:1094FC000000000000000000000000000000000060
:10950C00000000000000000043000000000000000C
:10951C00000000000000000000000000000000003F
:10952C0000000000000000004300000000000000EC
:10953C00000000000000000000000000000000001F
:10954C0000000000000000004300000000000000CC
:10955C0000000000000000000000000000000000FF
:10956C0000000000000000004300000000000000AC
:10957C0000000000000000000000000000000000DF
:10958C0000000000000000006B7600006D6B000016
:10959C00000000000A920000D491000042910000EB
:1095AC004291000042910000429100004291000063
:1095BC004291000042910000429100004291000053
:1095CC00FFFFFFFFFFFFFFFFFFFFFFFFFFFF00009D
:1095DC000100415343494900000000000000000015
:1095EC00000000000000000000000000000000006F
:1095FC0000004153434949000000000000000000F6
:10960C00000000000000000000000000000000004E
:10961C0000000000DD20000051220000F5250000B4
:10962C00A9330000BD410000B5200000000000007F
:040000030000268D46
:00000001FF
